:020000040800F2
:2000000000280020F10000083101000831010008310100083101000831010008000000007D
:200020000000000000000000000000003101000831010008000000003101000831010008D8
:200040003101000831010008310100083101000831010008310100083101000831010008D0
:200060003101000831010008310100083101000831010008310100083101000831010008B0
:2000800031010008310100083101000831010008E1040008310100083101000831010008DD
:2000A000310100083101000831010008310100083101000831010008310100083101000870
:2000C000310100083101000831010008310100083101000831010008310100083101000850
:2000E0003101000831010008310100085FF808F1002103E0094B5B58435004310848094B8B
:2001000042189A42F6D3084A02E0002342F8043B064B9A42F9D300F03DFA70471419000804
:2001200000000020C8020020C80200200C030020FEE7704703288CBF022000207047000091
:20014000034B1B689B7A13B10522024B1A607047040300200C0300200422014B1A60704757
:200160000C03002010B5002400F08EFC204B214A1B6812689C72D2791F495A721F4A0C60B8
:200180001368204623F4EC4323F0700343F400739BB21360136823F4E04323F040039BB2F0
:2001A00083F0100313600A68154B92B2134440225B001A6080220B689BB203F1005303F501
:2001C00040535B001A6000F04BFE0E4B20461B6893F8301000F09AFE204600F024FE01224E
:2001E000094B2046BDE810401A6001F027BB00BF0403002070020020505C0040005C004003
:2002000004300020DC0200200C030020014901F027B900BF78020020014901F021B900BF15
:2002200070020020054B1B689B78072B04D8044901EBC30101F014B900207047040300207F
:2002400088020020014901F00BB900BF8002002038B5174D04462A68127802F07F02212A1F
:2002600001D002201CE000F0A7FC0028F9D0601E0428F6D801A353F820F000BFA302000828
:20028000A7020008AB0200086302000891020008084B00242A682046936154829847204672
:2002A00038BD054BF5E7054BF3E7054BF1E700BF04030020CD0A0008FD0A0008250B0008BF
:2002C000E50A000808B5074B1B681B7803F07F03212B01D0022008BD00F06EFC0028F9D03E
:2002E0000020F8E704030020704770477047704770477047704770477047000037B5194C18
:200300000C20256800F074FB054045F4803500220C211548256000F0A9F900230193019B7C
:20032000B3F5007F1BD30C20256800F061FB054045F48025256000F06DFB0C4BC2B2186060
:200340000B4BC0F3072083F8292083F82A00094B5A71987103B0BDE8304000F0B1BE019B19
:200360000133DBE70408014000080140C802002094000020D3000020044A13689BB243F017
:200380000C0313600322024B1A607047405C00400C0300204FF6FB72034B19680A401A60E8
:2003A0004FF43F421A607047405C004010B51D4C072818BF20702378052B06D8DFE803F045
:2003C00003070B101823FFF7E5FF062306E0FFF7E1FF042302E0022363700323237006E05E
:2003E0006378013BDBB263706378002BF1D010BD0D4A13689BB243F010031360052323705F
:200400000A236370F3E76378013BDBB263706378002BECD14FF6EF73034A11680B4013609D
:20042000D3E700BFCE020020405C004001220020054B06491A60064A186010604FF4E0526E
:200440000A801A60704700BF405C004008030020445C004001220020034B1A60034A106073
:2004600003221A60704700BF405C0040445C0040FFF7F0BF07B5044B01A8019300F0FCF9D9
:2004800003B05DF804FB00BF1400000110B5002400F0CCFA084B1B689C72FFF7C7FF074BF0
:2004A000074A1C604FF43F431380064A1360FFF7E1FF054B1C6010BD04030020445C0040DE
:2004C00008030020405C00400C030020142307B501A8019300F0D0F903B05DF804FB0000F6
:2004E00070B5274D274C2B68274E9BB22380238832881340590505D54FF6FF332B60234B98
:200500005B689847228833881A40920444BF4DF6FF722A6022881340DB0405D54EF6FF7337
:2005200000202B60FFF742FF238832881340180504D5FFF721FF4FF2FF732B602388328872
:200540001340990507D54FF6FF5311492B600B780133DBB20B7023881A40D20505D54FF698
:20056000FF6307202B60FFF721FF2388328813401B0403D5BDE8704000F0E8BC70BD00BFCD
:20058000445C0040CC020020080300200000002010030020F7B500F0A3F800F0C5F800F03B
:2005A000F3F8FFF7ABFE00F009F900F041F90128044614D0022821D00023294800930522D5
:2005C0004FF4A0230D2100F063F8264800F004F9F0B100F055F8041E18BF012408E000233A
:2005E000052200930D214FF4A0231D4800F050F800252E461A4F052D11D984B91A4800F0C3
:20060000EBF8D8B1184800F07FF9002003B0F0BD154800F0E1F80028DBD10124E8E74FF4F5
:20062000801301220D213846009600F031F800F0DDFB08B100F0E0FB0135DCE7094800F023
:20064000CBF808B10748DEE74FF4A02305220D210090034800F01CF800F06AF9D5E700BF02
:20066000001001400050000800200008B2FA82F2012352098B40120103FA02F20261704721
:20068000024B1868C0F38000704700BF081401402DE9F8439DF820901446C9F10105EDB238
:2006A00006460F4698462A46013CE4B2FFF7DEFFFF2C10D1BDE8F88300BF013B002BFBD187
:2006C0004A4639463046FFF7D1FF43462BB92A4639463046E8E74346F0E700BF013BF5E7F7
:2006E0000D4B0E491A6842F001021A6008680C4A02400A601A6822F0847222F480321A60DC
:200700001A6822F480221A6000220B6823F4FE030B60044B1A6070470010024004100240E5
:200720000000FFF808100240154B1A6842F001121A601A689003FCD51221124A1160A2F649
:20074000FC72116841F4E81141F480611160196841F080711960196811F0407FFBD011685C
:2007600041F00201116011680907FCD59A6942F4FE729A61DA6942F40002DA61704700BFAA
:200780000010024000200240094A136823F4706343F4806313604FF48022064B1A60064A60
:2007A000136823F4700343F480131360704700BF001401401014014004100140054B1A68A0
:2007C000D1075EBF1A6842F001021A601A689207FCD570470010024003680348184000F1FF
:2007E00060435842584170470000FE2F034A43681060026882F30888184700BF08ED00E075
:20080000084AD36943F0C053D361074B1A6842F480721A60054A10851A6822F480721A6072
:20082000704700BF0010024000700040006C004044F24C210E4B10B5DA6942F0C052DA6111
:200840000C4A128D92B28A4219460DD044F24D239A420BD102240020FFF7D2FFCB6923F0A5
:20086000C053CB61204610BD0124F4E70024F9E700100240006C0040184B30B5DA680F2447
:20088000D243C2F30222C2F1040124FA02F2FF24437803FA01F18378134002780B4302F0CB
:2008A000FC0101F1604101F5614102F00300D1F80053C0001B0183406B4004FA00F0034084
:2008C0006B40C1F800330123510902F01F0203FA02F2034B43F8212030BD00BF00ED00E0BC
:2008E00000E100E04FF0FF32064BC3F88020C3F88420C3F88021C3F88421042243F8F02C83
:20090000704700BF00E100E0802210B50446074B1A60FFF7DBFDFFF7E5FFFFF7A9FDFFF7E9
:20092000DFFE2046BDE81040FFF760BF10200240024B034ADA6000BFFDE700BF00ED00E0F5
:200940000400FA050A4B10B51A6802221A60094A11461468E407FCD4074A106042221A60DA
:200960000A6812F00102FBD101201A6010BD00BF102002400C2002401420024073B501246A
:200980008BB200930B0C01930E4B1A681C600E4C25462668F607FCD4019CA4B244802C681A
:2009A000E607FCD4009CA4B204802C68E407FCD422F001021A600068431A5842584102B07C
:2009C00070BD00BF102002400C2002408022014B1A60704710200240034B044A1A6002F1B1
:2009E00088321A60704700BF04200240230167450F230728C8BF0838800003FA00F0C0437F
:200A000070470000024B188800F5003080027047E0F7FF1F044B1B88802B8CBF4FF4006054
:200A20004FF48060704700BFE0F7FF1F002302210C4A137053709370D370117153710A4A66
:200A40000A4913600A4A13800A4A11600A4A01F5884111600321094A1370094A1170094A7F
:200A600013707047110300201C0B0020000C0020180B0020C0020020C4020020200B00203F
:200A8000D002002017030020002210B50D4B0E4C197922600129C8B208D1022119711A70C9
:200AA000FFF720FFBDE81040FFF7E4BC10F0FD0F06D0022119711A70BDE81040FFF738BF9B
:200AC00010BD00BF110300201C0B002020B90122024B1B681A8270470148704704030020C9
:200AE0001503002020B90622024B1B681A827047014870470403002011030020064B1A686C
:200B0000538A28B9D188CB1A1382044B1980704703481844704700BF04030020180B00201E
:200B200018030020074B19684A8A20B9064B1B889B1A0B827047054B1868054B1B6818440E
:200B40001044704704030020180B00201C0B0020C00200202DE9F041134B144D1B782C68CA
:200B6000022B04F100640CBF04F5A04404F500542046FFF7E7FE0026DFF838800C4F3B88E6
:200B80009BB2B34208DC3B882A689BB213442B6000233B80BDE8F081A01958F8041BFFF799
:200BA000EDFE0436EBE700BF200B00201C0B0020180B002018030020012000227F49F8B5B7
:200BC0007F4C087025792270022DEBB264D108707C490968487801282FD1C888002800F0A2
:200BE000D0807948097B026003220129227105D0022918D00A23237122700FE07349744A78
:200C00001160744A1370FFF7D9FDFFF7E5FE7248FFF798FE44F24D20FFF7F2FD2078B0FA6D
:200C200080F04009F8BD6B4B1A70694B6A4A1A60FFF7C4FDFFF7D0FEECE7022823D109238C
:200C4000CA882371654B66481A801A8892B202801B884A889BB253435B4A13600B7B012B2C
:200C600006D0022B0CD00A23237103232370D5E7574B564A1A60FFF7C5FE5A4B1860CDE719
:200C8000534B554AF6E70628B5D0032801D12371C4E7052831D1FAE7032B0BD1494A126824
:200CA0005278032A04D105232371FFF753FFB5E7052AEFE7042B08D14B490878022801BFBD
:200CC000032362700B700523E1E7052B19D13D4B1A685378012B08D1D3880BB10323D6E7C3
:200CE00006232371FFF772FE98E7062B01D10223CDE7032BFBD0052BF9D00A2323710F2391
:200D0000B4E7062B08D12F4909684978032901D1082370E70529BDE7072BF9D0082BB6D07E
:200D2000092B39D1274B1A685378022B2DD1D18839B32A4852880388234D9BB25343244EAA
:200D40002B603368274FD5F800E00288734492B2D7F800C013446345214A04D803889BB218
:200D60001380092393E73B6830682D6828441B1A9BB2138013889BB29942B8D800231380E0
:200D8000B5E70A232371092370E7062BAFD0032BE7D0052BB1D1E4E70A2BAED1094B1B68D6
:200DA0005B78032B01D10A2371E7052BFBD0042BA3D102232371002358E700BF1703002029
:200DC00011030020040300201C0B002000500008C0020020200B0020002000081A0B00207F
:200DE000180B0020C4020020D0020020014B1878704700BF1703002000BFFDE7800000F138
:200E0000804000F5B8400368CA0623F4E04323F040039BB248BF83F010038A0648BF83F076
:200E2000200303607047800000F1804000F5B840036823F4804323F070039BB283F4405335
:200E400003607047800000F1804000F5B840036823F4E24323F070031B041B0C03607047CD
:200E6000FFF7F0BF800000F1804000F5B84003685B0409D5036823F4E04323F070031B04BD
:200E80001B0C43F4804303607047800000F1804000F5B84003685B0609D5036823F4E043AA
:200EA00023F070031B041B0C43F0400303607047064B1B689BB203EBC00000F1005000F5D1
:200EC00040504000006880B2704700BF505C0040054B1B689BB203EBC000044B03445B0087
:200EE000186880B2704700BF505C004004300020044B1B689BB203EBC000034B03445B00CD
:200F000019607047505C0040023000200D4B0E4A1B683E299BB203EBC00002444FEA42020B
:200F20000AD94B09C80604BF03F1FF339BB29B0243F40043136070474B08C90748BF0133D7
:200F40009B02F7E7505C0040063000202DE9F843DFF86481DFF86491D8F800304F4A99B217
:200F60001B04118052D547F6FF73C8F80030138803F00F0389F80030002B63D1484C494E20
:200F80002368494D03F4405333802368474F03F030032B8023683B409BB283F40053236061
:200FA000236823F4E04323F040039BB283F020032360138813F0100F236829D123F4E14333
:200FC00023F070031B041B0C236000F053FC236832883B409BB2D70448BF83F480539604B0
:200FE0002F4A48BF83F40053136013682A8823F4E04323F040039BB2D40648BF83F01003C3
:201000009006274A48BF83F020031360BDE8F883190601D52368D1E71A0508D5236823F0C7
:2010200070031B051B0D236000F048FACFE71B0492D5236823F070031B051B0D236000F038
:201040009DFBC4E79A0002F1804202F5B842146821040AD51168013B21F070010905090D32
:201060001160134A52F82330984722067FF574AF99F80020930003F1804303F5B8431968F8
:20108000013A21F4E14121F070010904090C1960084B53F8223098475EE700BFCC02002000
:2010A000005C0040D2020020D40200208FBFFFFF780000205C000020445C0040E002002068
:2010C000064B074A0749136002221A72064B074A1360074A1B681160184700BFE40200207D
:2010E000040300203800002000000020DC0200200003002010B5064C18B9012223681A82FE
:2011000010BD044B1B681B68984720680A30F7E7040300200003002010B5064C18B90122D9
:2011200023681A8210BD044B1B689B68984720680C30F7E704030020000300201F4B10B5EC
:201140001968034600201BB9022218460A8210BD1B4C20800B78224613F07F0312D1497AD9
:201160008C0644BF02231370137848064CBF23F0010343F001031370124B1B681B6998473A
:201180000F48E4E7012B17D0022BE0D1097901F00F039B0003F1804303F5B84309061B68E0
:2011A00005D503F03003102BE6D10123E3E703F44053B3F5805FF7E72046C8E70403002024
:2011C0000A030020000300202DE9F843234FDFF8A0803D682C8AD4B92E7A042E17D12049F2
:2011E0000B78012B0ED11F4B1A681F4B92B213445B001C6030230C70A8F800303B681E72C7
:20120000BDE8F88310230726A8F80030F6E7AA8AAB69944294BF04260226944228BF1446C7
:201220002046984781460020FFF742FE22460146484600F04DFB21460020FFF759FE2B8A4E
:201240006A8A1B1B2B82302314444FF44052A8F80030064B6C821A80D0E700BF04030020F1
:20126000210B0020505C004002300020D2020020D402002010B50A4B0A491B6849789A7837
:2012800091420AD3DC7844B9998831B99A72064B1B685B689847204610BD0224FBE700BFC6
:2012A00004030020340000200003002038B50E4A0E4D12682B6892699978187990472B68DC
:2012C0009A7A7AB170B95A7962B9DC7854B9084B1B68DB6898472B681A79DA729A781A734E
:2012E000204638BD0224FBE7DC020020040300200003002070B52D4B1D682B7813F07F03F9
:2013000005D16A7A22F020026A72184670BD022B49D16A88002AF8D16A79002AF5D12979D7
:20132000234E21F08000840004F1804404F5B8442268367849B20029B4BF02F0300202F490
:2013400040528642E1D9002ADFD0AA7A002ADCD00029236811DA03F03003102B07D1C4B258
:201360002046FFF792FD30212046FFF747FD114B1B685B6998470023C7E703F44053B3F50C
:20138000805FF4D10C4D58B90C4B93F83010FFF7BDFD23682B409BB283F440532360E6E7D0
:2013A000FFF760FDF5E70223AFE700BF0403002034000020000300208FBFFFFF000000207A
:2013C00038B51B4B1B4D18682D78017921F08004A30003F1804303F5B8431A6849B200292B
:2013E000B4BF02F0300202F44052A5421DD94488DCB9D2B1827AC2B11A680029B5BF22F469
:20140000E04222F4804222F0400222F07002B5BF92B292B282F0100282F480521A60064B67
:201420001B689B699847002038BD0220FCE700BF04030020340000200003002008B5064BC1
:201440001A68537A43F020035372044B1B68DB699847002008BD00BF04030020000300203F
:20146000054B10B51C68628A18B98B889B1A238210BD08681044FBE70403002008B50B4BFC
:20148000002093F83010FFF741FD094B1B68187A082806D14FF48052064B1A801022064B3A
:2014A0001A80A0F109035842584108BD0000002004030020D2020020D402002073B5974DC0
:2014C000974B2A68974C92B213445B001A682368197A09290FD092B2520002F1804202F5CC
:2014E000C042117819705178597091885980118999809289DA8001221A72DA885E78002A1B
:2015000064D11A7812F07F024DD1092E03D1FFF7B1FE40BB16E0052E20D193F90220002AC6
:2015200007DA08232268137202B0BDE87040FFF7A5BFDA78002AF4D19A88002AF1D19B7ACB
:20154000002BEED12A68784B92B2134400225B001A603022754B1A800623E3E7032E14D105
:201560009A78012A08D0724B30461B685B699847032828D10923D5E79A88002AF3D15B7A0C
:201580009A06F0D5FFF75AFFC3E7012EEBD19A78012AE8D19A88002AE5D15B7A9B06E2D5DD
:2015A000FFF7A8FEB5E7012A04D10B2EDBD1FFF77DFEAEE7022AD6D1012EF1D0032ED2D171
:2015C000FFF7FEFEA5E70028BCD0AAE7062E17D11A7855065ED1DB78554A012B126803D1A4
:2015E000D369002B56D01EE0022B01D1136AF8E7032B01D1536AF4E7212B4BD1936AF0E731
:20160000002E54D15988002944D15A6822F0FF02B2F5003F3ED11A7812F07F0215D19B8870
:20162000002B37D1434B0025226828465582936198474FF6FF7123681A8A8A4234D0022D3F
:2016400001D0002A56D108222FE0012A0AD1384A1879126892699047E0B923689B7A002B66
:20166000E0D117E0022A15D11A7902F00F018B00100603F18043304803F5B8431B6800785D
:201680004CBF03F0300303F44053884202D912F0700FE4D0264B22681B6850781B6998470C
:2016A00003280546C5D1236809221A723CE7082E04D11B785B06EDD1204BB4E70A2EE9D104
:2016C0001A7802F07F02012AE4D19A7A002AE1D059880029DED15A6822F0FF02B2F5803F42
:2016E000D8D1134A18791268926990470028D1D1134B98E793F90010002934DAD9880C48D8
:2017000001910068019D90F83040AA42204619D9019A1A829882FFF757FD05E7505C004082
:20172000043000200403002002300020D4020020DC0200203D11000834000020F510000831
:20174000191100088A42E5D2A24203D20021094A1170DFE7B2FBF4F104FB1122002AD9D1C8
:201760000121044AF4E703221A724FF44052024B1A80D9E6210B0020D2020020F8B5294E8E
:201780003468237A032B01D0052B43D1A369B3B1258A0DB3A28A954228BF1546284698475C
:2017A000238A07465B1B2382638A00202B446382FFF78EFB2A460146384600F098F8238AD2
:2017C00053B100214FF44052174B08461A80FFF78FFB3022154B1A80218AA38A32688B42BA
:2017E00008D803231372137A32681372BDE8F840FFF744BE09B10523F4E7062313720C4B1B
:2018000018680C4B80B203445B0019603021074B1980E8E7072B03D1074B1B68DB6898479C
:201820000823E1E704030020D2020020D4020020505C004002300020DC02002030B5002261
:2018400048F68F75094B1C78A24204D3084B40F08000186030BD930003F1804303F5B843FE
:2018600019682940114319600132EDE7340000204C5C004010B5134C23681A7A022A01D02E
:20188000042A09D1FFF7A0FC23681B7A22681372BDE81040FFF7F2BD062A10D15A78052AD3
:2018A00009D11A78520606D19878FFF7C7FF064B1B681B6A9847054B1B689B6898470823A9
:2018C000E4E700BF0403002000030020DC02002001F10051013201F540515210490002B9D3
:2018E000704730F8023B013A21F8043BF7E7002310B501F10051013201F5405152104900CB
:201900009A4200D110BD51F8234020F813400133F6E700008D0400086501000833010008E2
:20192000ED02000851020008C5020008350100080D02000819020008250200084502000890
:20194000000000004000000001010000EF02000841010008F1020008F3020008F50200080B
:20196000F7020008F9020008E902000859010008EB020008EB020008EB020008EB0200083A
:20198000EB020008EB020008EB020008EB020008EB020008EB020008EB020008EB0200089F
:2019A000EB020008EB02000809022D0001010080320904000000FE0102040904000100FE33
:2019C0000102050904000200FE010206092103FF00000810011201000100000040AF1E0380
:2019E00000010201020301092103FF00000810018003530054004D003300320064007500E3
:201A000069006E006F00200062006F006F0074006C006F006100640065007200200076009F
:201A200031002E003000200020004500520052004F0052002E002000550070006C006F005F
:201A400061006400200074006F002000520041004D0020006E006F00740020007300750045
:201A6000700070006F0072007400650064002E006C03530054004D00330032006400750099
:201A800069006E006F00200062006F006F0074006C006F006100640065007200200076001F
:201AA00031002E00300020002000550070006C006F0061006400200074006F002000460089
:201AC0006C0061007300680020003000780038003000300035003000300030006C03530077
:201AE00054004D00330032006400750069006E006F00200062006F006F0074006C006F0012
:201B000061006400650072002000760031002E00300020002000550070006C006F006100C3
:201B20006400200074006F00200046006C00610073006800200030007800380030003000D0
:201B400032003000300030000403090414034D00610070006C0065002000300030003300F6
:201B600010034C004C004D00200030003000330012034C006500610066004C00610062001E
:201B800073000000940000202D000000C100002012000000D30000200900000034020020AC
:201BA000040000005C0200201200000038020020140000004C02002010000000DC000020A9
:201BC000800000005C0100206C000000C80100206C000000000C002000500020FFFFFFFFAF
:201BE000FFFFFFFFFFFFFFFFFFFFFFFFFFFFFFFFFFFFFFFFFFFFFFFFFFFFFFFFFFFFFFFF05
:201C0000000C00200000000000000000000000000000000000000000000000000000000098
:201C20000000000000000000000000000000000000000000000000000000000000000000A4
:201C4000000000000000000000000000000000000000000000000000000000000000000084
:201C6000000000000000000000000000000000000000000000000000000000000000000064
:201C8000000000000000000000000000000000000000000000000000000000000000000044
:201CA000000000000000000000000000000000000000000000000000000000000000000024
:201CC000000000000000000000000000000000000000000000000000000000000000000004
:201CE0000000000000000000000000000000000000000000000000000000000000000000E4
:201D00000000000000000000000000000000000000000000000000000000000000000000C3
:201D20000000000000000000000000000000000000000000000000000000000000000000A3
:201D4000000000000000000000000000000000000000000000000000000000000000000083
:201D6000000000000000000000000000000000000000000000000000000000000000000063
:201D8000000000000000000000000000000000000000000000000000000000000000000043
:201DA000000000000000000000000000000000000000000000000000000000000000000023
:201DC000000000000000000000000000000000000000000000000000000000000000000003
:201DE0000000000000000000000000000000000000000000000000000000000000000000E3
:201E00000000000000000000000000000000000000000000000000000000000000000000C2
:201E20000000000000000000000000000000000000000000000000000000000000000000A2
:201E4000000000000000000000000000000000000000000000000000000000000000000082
:201E6000000000000000000000000000000000000000000000000000000000000000000062
:201E8000000000000000000000000000000000000000000000000000000000000000000042
:201EA000000000000000000000000000000000000000000000000000000000000000000022
:201EC000000000000000000000000000000000000000000000000000000000000000000002
:201EE0000000000000000000000000000000000000000000000000000000000000000000E2
:201F00000000000000000000000000000000000000000000000000000000000000000000C1
:201F20000000000000000000000000000000000000000000000000000000000000000000A1
:201F4000000000000000000000000000000000000000000000000000000000000000000081
:201F6000000000000000000000000000000000000000000000000000000000000000000061
:201F8000000000000000000000000000000000000000000000000000000000000000000041
:201FA000000000000000000000000000000000000000000000000000000000000000000021
:201FC000000000000000000000000000000000000000000000000000000000000000000001
:201FE0000000000000000000000000000000000000000000000000000000000000000000E1
:2020000000500020AD4E00087151000875510008795100087D51000881510008D151000809
:20202000D1510008D1510008D1510008D1510008D1510008D1510008D151000829580008F1
:20204000D1510008D1510008D1510008D1510008D1510008D15100081D550008235500088A
:20206000295500082F550008355500085D5300086D5300087D5300088D5300089D53000884
:20208000AD530008BD53000829520008D15100082D5D0008D1510008D15100083B550008F5
:2020A000315A0008555A0008795A0008AD5A0008FD5A0008095B0008155B00080D5600083E
:2020C000255600081956000831560008D1510008D1510008E95B0008015C0008195C0008F5
:2020E00043550008D1510008D151000810B5054C237833B9044B13B10448AFF300800123AA
:20210000237010BD38070020000000000C94000808B5064B1BB106480649AFF30080064871
:20212000036813B1054B03B1984708BD000000000C9400083C07002038070020000000005E
:2021400090F900308B4205D000230022436002814281C360017070472DE9F7430446476862
:202160000846884606F0BEFA0146384606F00EFBE16806F003FA0021064606F0C3FCB0B112
:20218000304605F0F3FA2E49054606F0B1FC50B928464FF0434106F0A1FC30B9284606F068
:2021A000BBFCC5B204E07F2502E0802500E0054668B206F097FA0146304606F0DDF92389E1
:2021C000E06033B1984528BF9846C8EB030323811BE06689BEB1B04528BFB046C8EB0608F0
:2021E000404606F07FFA0146384606F0CFFA8146304606F077FA0146484606F07BFBA4F8E5
:202200000A80606001E000236360237838465D4300218DF8045006F04DFC48B960680021D1
:202220004FF0010506F046FC00B90546EDB200E000259DF8040040EA052003B0BDE8F083C6
:202240000000FE4208B504F0A9FF003018BF012008BD08B504F0A2FF003018BF012008BDB9
:2022600038B5094C04F108056078002104F0CAFE6078002104F0A8FF14F8010F052104F09B
:20228000C1FEAC42F0D138BD0F00002038B5074C04F108056078002104F0B4FE14F8010FAF
:2022A000002104F091FFAC42F4D138BD0700002008B5FFF7EBFFFFF7D3FF002307490022B0
:2022C0005A5407495A5407495A540133082BF5D1BDE808404FF4FA7004F0A6BFF00800201C
:2022E00094070020FC0800202DE9F0410025384E0121384C705D04F067FF4FF42F7004F06A
:20230000A8FF2078FFF7A5FF80466078FFF7A1FF0746A078FFF79DFF800040EA4707E07869
:20232000FFF797FF47EA0807FFB247EAC000C7B22079FFF78EFF47EA0010C7B26079FFF711
:2023400088FF47EA4010C7B2A079FFF782FF47EA8010C7B2E079FFF77CFF47EAC010C4B2F1
:202360000021705D04F030FF1B4BEA5C1E46A24206D05C55194B01221A70194A12685A8009
:202380000135082DB3D115480378D3B1144B1A684388D31A142B14D9002300210A46B45C89
:2023A0001C4104F00104944001322143082AC9B2F5D10C4AD1540133082BEED100230370B2
:2023C00002E0012004F030FF0120BDE8F08100BF080000201000002094070020F8080020AE
:2023E00044120020F008002008B5FFF761FF024B00221A705A8008BDF808002008B5302077
:2024000004F0CCFEC0B208BDE92910B50B46044624D004D8C1290ED0E82913D034E0F42998
:202420002DD031D3A1F1F802042A2DD8BDE81040C06802F047B90068002380F861300368CE
:202440001B6913E0FFF7DAFF012804D12068202103681B690AE0A06809210BE0FFF7CEFFB6
:20246000012805D12068B02103681B69984710BDA0680A210022BDE8104002F02FB9002322
:202480008374C385838510BD2068D9B202681269904710BD38B5084D0C4635F8111021B9D0
:2024A0001146BDE83840FFF7AFBFFFF7ADFF002325F8143038BD00BF7008002073B502EBBD
:2024C000C101827C1E460446C9B26E4B3AB101EB821233F812506C4B01225A5404E0027C78
:2024E00001EB821233F812504FF6FF739D4200F0C680F42D05D0FE2D03D0E37D012B00F093
:20250000BE80012E05D1614B33F811200AB923F81150F92D60D00DD8E92D3BD004D8C12D0B
:2025200015D0E82D1FD09BE0F42D00F08D80F82D4DD095E0FC2D67D004D8FA2D5BD0FB2DAC
:202540004FD08DE0FE2D62D0FF2D67D088E0012E40F08D80206829460368DB68984723684C
:2025600083F861608BE00191FFF748FF012801990BD1012E04D1206820210368DB6815E0D6
:20258000002E7CD12046202274E0012E70D1A068092116E00191FFF731FF012801990CD1D4
:2025A000012E05D12068B0210368DB68984766E0002E64D12046B0225CE0012E58D1A068B3
:2025C0000A21324602B0BDE8704002F087B8012E4ED1E0686F2112E0012E49D1E0687021E6
:2025E0000DE0012E44D1A38A13B1E068E22106E0E068E92103E0012E3AD1E068EA2102B014
:20260000BDE8704002F05AB8012E31D1EDE7012E35D1E37D83F00103E37530E0012E2ED1BA
:20262000A37D1B480133DBB2022B88BF0023A37504F03AFCA27D174B082033F8121002B0D5
:20264000BDE8704004F0C2BC012E04D1638DB3B9A674E58513E096B9A674E685A6850EE0EF
:20266000012E04D12068E9B20368DB689EE736B920462A4602B0BDE87040FFF70BBF02B0C2
:2026800070BD00BF009D00080C0800207008002008080020889B000870B50E4BA2B05B5CFB
:2026A00006461341DB070D46144611D50A2301FB033313440133009307492A46234602A8B5
:2026C00006F052FB3046294622460123FFF7F6FE22B070BDF00800208E9B0008F0B50F4B15
:2026E000A3B05B5C0746134113F001060D46144611D10A2201FB02222244013200920849CE
:202700002A46234602A806F02FFB3846294622463346FFF7D3FE23B0F0BD00BFF00800202A
:20272000A19B00082DE9F84F8046FFF7DDFD0024154B5FFA84F9E75C144B14F803B09A46C7
:2027400097EA0B0B04D10134082CF1D1BDE8F88F0025012616EA0B0F0ED03E4240464946DD
:202760002A4602D0FFF798FF01E0FFF7B7FF1AF8043073400AF804300135EDB27600082D4E
:20278000F6B2E7D1DFE700BFF0080020FC08002010B50024044B0421185D013404F032FCEF
:2027A000112CF7D110BD00BF1800002038B51E2004F04FFD00242546154B185DFFF742FD4C
:2027C00080F00100C3B2A3400134112C45EA0305F2D110490B68AB420F4B05D001221A702F
:2027E0000E4A0D6012685A801B780B4A5BB10B4B18685388C31A052B05D9094B09681960F2
:202800000023137002E0012004F00EFD012038BD1800002068080020A407002044120020F1
:20282000A007002010B50446FFF7B2FFA06840F2FF1101F062FFA06840F2FF1101F07AFFCB
:20284000024B00221A705A8010BD00BFA407002081422EBFC0EB01004042C1EB000070470D
:2028600010B51446FFF7F4FFA04228BF204610BD38B50B4B04461D68038913B94FF47A73BA
:2028800008E0006829464FF47A72FFF7E9FF63681844430863604FF47A732560238138BDE9
:2028A0004412002003898B428CBFC1EB030300230381038913B143681944416070470000F5
:2028C00008B5038953B1406830B105F007FF0146034806F00FF808BD014808BD002008BDE0
:2028E00000007A4443780BB10123837070470023437083708088C01A18BF01207047EC2966
:2029000038B504460B465DD018D8852935D00BD8812932D001D8802903E0822900F0BB8095
:20292000842900F0AE80CBE0872900F0BE80C0F0B280EA292DD0EB2934D0C1E0F12900F08E
:20294000828007D8EE2956D045D3EF295FD0F0296DD0B5E0F72900F0918004D8F5297ED0A6
:20296000F6297FD0ACE0FD2900F0A480B1F5807F40F0A6800023838238BDE58B002D40F03E
:20298000A4802068D9B20268126990476584258438BDFFF733FD01280DD12068DA210368A2
:2029A0001B6985E0FFF72AFD012804D12068D92103681B697CE0A06840F2FF11BDE83840DF
:2029C00001F0B8BEFFF71AFD01280DD12068D82103681B696CE0FFF711FD012804D1206836
:2029E000D72103681B6963E0A06840F2FF11BDE8384001F082BEFFF701FD012804D120689B
:202A00006A2103681B6953E0A06802210AE0FFF7F5FC012804D120686B2103681B6947E0E5
:202A2000A06803210022BDE8384001F057BEFFF7E5FC012804D12068752103681B6937E02C
:202A4000A0680121EEE7FFF7D9FC012804D12068692103681B692BE0A0680421E2E7406804
:202A6000012129E0436B9B781BB94068042101F021FF606BBDE83840FFF739BF4068022117
:202A80001AE0258B0DBB2068D9B2026812699047A583658338BDA58CBDB92068D9B20268CC
:202AA000126990472585E58438BD006803681B69984738BD40680421BDE8384001F03EBFB9
:202AC0002068D9B202681269904738BD38B5084D0C4635F8111021B91146BDE83840FFF70C
:202AE0000EBFFFF70CFF002325F8143038BD00BFA8070020F8B5837C164604460F46A54A6B
:202B000003B9037C03EB03133B4432F813504FF6FF739D4200F07881E37D012B00F074817A
:202B2000012E05D19C4B33F817200AB923F81750EC2D00F0848018D8852D3CD00BD8812DB6
:202B400039D001D8802D03E0822D00F03381842D00F0248148E1872D00F03781C0F02A818A
:202B6000EA2D36D0EB2D4CD03EE1F12D00F0E7800AD8EE2D00F0998079D3EF2D00F0AD80E5
:202B8000F02D00F0C1802FE1F72D00F0FE8006D8F52D00F0EE80F62D00F0F08024E1FD2D35
:202BA00000F01A81B5F5807F40F01E81012E40F02481A582F8BD012E40F01E81E38B002B9B
:202BC00040F022812068E9B20368DB6898476584F8BDFFF713FC01280DD1012E04D120683C
:202BE000DA210368DB6805E1002E40F00D8120463946DA2204E1002E00F0FF80A0680021CE
:202C000019E0FFF7FBFB01280DD1012E04D12068D9210368DB68EDE0002E40F0F58020468E
:202C20003946D922ECE01EB920463946EB22E7E0A06840F2FF31BDE8F84001F07BBDFFF758
:202C4000DDFB01280DD1012E04D12068D8210368DB68CFE0002E40F0D78020463946D8221F
:202C6000CEE0002E00F0C980A068002119E0FFF7C5FB01280DD1012E04D12068D721036871
:202C8000DB68B7E0002E40F0BF8020463946D722B6E01EB920463946ED22B1E0A06840F2B3
:202CA000FF31BDE8F84001F028BDFFF7A7FB01280DD1012E04D120686A210368DB6899E054
:202CC000002E40F0A180204639466A2298E0012E40F09380A068022146E0FFF78FFB012820
:202CE0000DD1012E04D120686B210368DB6881E0002E40F08980204639466B2280E0012E67
:202D00007BD1A06803212FE0FFF778FB01280CD1012E04D1206875210368DB686AE0002E75
:202D200072D12046394675226AE0012E03D10121A0680A4619E020463946F02260E0FFF7E7
:202D40005DFB01280CD1012E04D1206869210368DB684FE0002E57D12046394669224FE02D
:202D6000012E4AD1A06804213246BDE8F84001F0B5BC012E40D16068314631E0012E3CD159
:202D8000636B00225E709A80F8BD012E34D16068022125E0E09B0008A8070020012E2CD104
:202DA000238B002B30D12068E9B20368DB689847A583F8BD012E20D1A38C2BBB2068E9B254
:202DC0000368DB6898472585F8BD012E15D1206829460368DB680DE0012E0DD16068042166
:202DE000BDE8F84001F0A5BD012E05D12068E9B20368DB689847F8BD36B9204639462A46F5
:202E0000BDE8F840FFF762BEF8BD00BF2DE9F8430646114FFFF7CAFC10493A680B68894655
:202E200092EA030816D00025012414EA080F0BD0D9F8002030462240294618BF0122FFF7C3
:202E400059FE3B6863403B600135EDB2112D4FEA4404EAD1BDE8F88354070020A007002089
:202E600073B5054672B6426B002354789380374A84F0010411781646A14205D0344A13815F
:202E80009382344A137009E0314895F83810FFF709FD314895F83810FFF704FD012C3470D3
:202EA0002E4E27D12E4C95F838102046FFF754F995F83810ADF8000004F11000FFF74CF9EC
:202EC000ADF80400C2B29DF801009DF80010234628B10020606100241C835C83D8619DF807
:202EE000050028B10020002458611C835C83D861002417E0174B71781A780A44D2B254B270
:202F0000022194FBF1F4E4B2C4EBC41102EB41021A702CB1686BFFF7E5FC0022114601E065
:202F20002246214600233370737062B609B902B94CB16342686849B252B25BB202B0BDE8AF
:202F4000704001F0D5BC02B070BD00BF04080020EC0700209C070020F80700200508002053
:202F6000CC070020104A08B5104B11681868FF221960FFF775FC0E4BC0B298635B6B80B234
:202F80009A8882428BBFC0EB0200002298809A800748FFF765FF0648FFF738FFBDE80840EF
:202FA0000348FFF7BFBB00BF441200206C0800205807002008B52B20022104F023F828208C
:202FC000022104F01FF82920022104F01BF82A20022104F017F82B200A49022203F0CEFF5E
:202FE00029200949022203F0C9FF28200749022203F0C4FFBDE808402A200549022203F049
:20300000BDBF00BF3134000891330008ED3200084D3200082DE9F041784F8CB03846784905
:2030200001F09CFC3846774901F09AFC7649384601F098FC642003F0C7FF744B00240360FD
:203040000225092344608DE82800714B064602941A68704906F14803083001F0D3FE6E4B0E
:2030600086F85A503360A6F8585006F151034FF0010886F86050694D736586F85B8086F829
:20308000618050202E6003F09FFF0D2214238DE80C00634B029406461A685E4900F14003EC
:2030A00001F0B0FE96F8403086F8484033640F2386F84530202386F846306FF07F0386F81B
:2030C0004730022386F84930082386F84A3086F84B4086F84C4086F84D4086F844404820B2
:2030E000AE6003F071FF05238DE808014D4B029406461A68474900F1410301F083FE86F808
:20310000404044206E6003F05FFF032300930193454B02941A6806463E4900F1400301F0BF
:2031200071FE336C062064F3172333642B68EE6083F8614003F048FF0470447084708480DC
:2031400068631C202C746C74AC74AC82AC75EC752C836C83AC83EC832C846C84AC84EC849C
:203160002C856C85AC85EC8503F02EFF2F494460034640224FF47A70196098601C745A613B
:203180009A612B63DB680790089305910A920B9205A9274ADB231F4806948DF8244001F06A
:2031A000C5FD244B97F874101A6801B9FEE7137B052BFAD11948FFF717F91848FFF732FB37
:2031C0001648FFF7F7FE3020022103F01BFFC821194803F077FE184803F066FE082007216D
:2031E00003F010FF0021082003F0F0FE4FF47A7004F01AF80CB0BDE8F08100BF5C0E002055
:20320000C29B0008CE9B0008D79B0008F0A30008E40100204C080020809F000858070020A4
:20322000E0010020E8010020C0010020A09F0008249C0008380600200808002008B504F055
:2032400017FEBDE8084004F0D5BA00002DE9F041224B234D5A78234C05F10C0701323846CA
:203260005A70FFF705FB012104F11000FEF768FF2846FFF725FB06463846FFF721FB314634
:203280000746304605F082FA39468046384605F07DFA0146404605F071F904F001FB124954
:2032A000804620F0004005F025FB414605F022FB80464146384605F069FA414607463046DD
:2032C00005F064FA6060288AFFF7B8FF05F0E0F880B2676120836083BDE8F08105080020EC
:2032E000EC070020CC0700200000F0412DE9F041234B244D5A78244C05F10C07013A38466D
:203300005A70FFF7B5FA4FF0FF3104F11000FEF717FF2846FFF7D4FA06463846FFF7D0FA03
:2033200031460746304605F031FA39468046384605F02CFA0146404605F020F904F0B0FADC
:203340001249804620F0004005F0D4FA414605F0D1FA80464146384605F018FA414607464C
:20336000304605F013FA6060288AFFF767FF05F08FF880B2676120836083BDE8F08100BF36
:2033800005080020EC070020CC0700200000F0412DE9F041224B234D1A78234C0132284603
:2033A0001A70FFF765FA01212046FEF7C9FE2846FFF786FA074605F10C00FFF781FA3946C7
:2033C0000646384605F0E2F931468046304605F0DDF90146404605F0D1F804F061FA13499F
:2033E000804620F0004005F085FA414605F082FA80464146384605F0C9F94146074630467F
:2034000005F0C4F90646A888FFF718FF05F040F880B26760208160816661BDE8F08100BF2D
:2034200005080020EC070020CC0700200000F0412DE9F041224B234D1A78234C013A28465A
:203440001A70FFF715FA4FF0FF312046FEF778FE2846FFF735FA074605F10C00FFF730FA9B
:2034600039460646384605F091F931468046304605F08CF90146404605F080F804F010FA1F
:203480001249804620F0004005F034FA414605F031FA80464146384605F078F941460746EC
:2034A000304605F073F90646A888FFF7C7FE04F0EFFF80B26760208160816661BDE8F081C4
:2034C00005080020EC070020CC0700200000F0410E4B10B54022002401210D485A6019702A
:2034E0005C70DC601C615C6103F0C8FC094B00221C81DC609C821C60074B5A601C815C8164
:20350000DA605A611C835C83DA6110BD4C08002008080020EC070020CC07002008B51E4962
:20352000422205F067FB1D4A0346917D90F82600014483F8261093F8360092F82210927AE5
:20354000014483F8361093F83D1098780A4483F83D20134A9178014499709278997A114431
:20356000997293F82D10114483F82D10997E1144997693F82210114483F8221093F8231073
:203580000A4483F82320074A12681A87064A1268A3F83F2008BD00BF009E00085C00002049
:2035A000300000208000002084000020064A00231360064A1360064A1360064A1360064BF7
:2035C000FF221A70704700BF1C0B0020140A0020100A0020080900200509002007B5074B9E
:2035E000074A1B680092074A0749019207484FF4807200F0C5FE03B05DF804FB100A0020B9
:2036000008090020050900201C0A00205C00002002F07F02212A13B514D199B9022805D0CD
:20362000222805D1094A03F0030313700C4600E00224074B1B6833B102A901F8010D0220B6
:20364000984700E00224204602B010BD04090020180A002037B502F07F02212A05460C46EA
:203660001AD1C9B9202807D021280BD10C480721224600F0C3FD06E009480721224600F04E
:2036800031FE00E00224074B1B6833B102A901F8015D0220984700E00224204603B030BD2D
:2036A00029000020180A002037B51A4D1A4C2A6802AB43F8042D04F118004FF48072174979
:2036C00000F02EFE019B164A2B6012689B1A154ADBB21268C2F58072934212D294F8223072
:2036E0009B0003F1804303F5B8431A6822F4804222F0700242F4004242F0800282F4405273
:203700001A60094B1B6813B101200021984703B030BD00BF1C0B00205C0000200C0900201C
:20372000140A0020800000200C0A0020034B002808BF40201881024B186070475C00002047
:2037400084000020002808BF402008B580B200F061FE024B1884024B186008BD5C00002049
:2037600080000020C20744BF034B1960830744BF024B1960704700BF0C0A0020180A0020D5
:2037800070B50C4629B31449144A0B6812680D469A1AD2B2C2F1FF02944201D9BAB114467A
:2037A000002291B2A14202F1010205D2465C0C49CE540133DBB2F4E72B600A4B1A781206B5
:2037C000FBD51B781B0604D5FFF708FF01E0104670BD204670BD00BF100A0020080900206E
:2037E0001C0A002005090020034B1868034B1B68C01AC0B2704700BF1C0B0020140A00206F
:203800000A4B10B51A680A4B1B689B1ADBB2994228BF194600238B4206D0064CA45C013286
:20382000C454D2B20133F6E7184610BD140A00201C0B00200C09002008B5FFF7E1FF104A09
:2038400013680344DBB213600E4A1268D31ADBB2402B13D80C4B93F822309B0003F180437E
:2038600003F5B8431A6822F4804222F0700242F4004242F0800282F440521A6008BD00BF45
:20388000140A00201C0B00205C0000200B4B10B51B6819440A4BC9B21B685B1ADBB2934202
:2038A00038BF1A460023934206D0064C645C0131C454C9B20133F6E7184610BD140A002092
:2038C0001C0B00200C090020024B187800F00100704700BF04090020014B1868704700BFB9
:2038E00029000020800000F1804000F5B840036823F4E04323F0400343F4004343F0800336
:2039000059400160704700000B4B1B685A8A20B90A4909888A1A1A8270470949096831B1E0
:20392000D8889B8A134498429CBF01230B70054B186800B1104470477C120020E00C002091
:203940004C0B0020D80C0020104B10B51B685A8A60B90F4CD98824888C4238BF21468A42EC
:203960003ABFC2EB01021A82188210BD0949096831B1D8889B8A134498429CBF01230B7046
:20398000054B186800B1104410BD00BF7C1200204A0B0020DC0C0020E40C00202DE9FF4135
:2039A000164B1C68227802F01F03012B21D1144B2179D3F800C0134BD3F80080002363455E
:2039C00017D058F82360376A8FB1B5788D420ED836782E44B1420ADA491BE578A378009502
:2039E000A588C9B20195E4880294B84702E00133E5E7022004B0BDE8F08100BF7C1200204D
:203A0000440B0020B80C00202DE9F341154B1C68227802F01F03012B1FD1134B2179D3F898
:203A200000C0124BD3F800800023634515D058F82360776A7FB1B5788D420CD836782E448A
:203A4000B14208DA491BE578A3780095A488C9B20194B84702E00133E7E7022002B0BDE888
:203A6000F08100BF7C120020440B0020B80C002010B50B4B1B689B7A1BB10A4B05221B6897
:203A80001A730024084B1B689C4208D2074B1B6853F824305B6903B198470134F2E710BD41
:203AA0007C12002038060020440B0020B80C002010B50024064B1B689C4208D2054B1B685F
:203AC00053F824309B6903B198470134F2E710BD440B0020B80C0020024B04221B681A73FF
:203AE000704700BF38060020012906D8044B1B79834294BF0220002070470220704700BF5E
:203B0000500B002030B5134B05461B689A78124B1B7893421CD9114C04EBC2018B889BB9D7
:203B200054F83200C45C0E4A59002CB1242B03D00A4454800133F5E78B1C0A49D8B2107001
:203B40008880A84228BF2846BDE8304002F0F2BD002030BD7C1200206801002048010020BB
:203B6000880000206C010020014902F0E3BD00BF20010020014902F0DDBD00BF2801002056
:203B800038B5154B00221B6801219A72134B4FF4E050196412490C681A645A6418644FF4ED
:203BA0003F405A64206018640E4B4FF48010186014460D460C4B1B689C4208D20B4B1B6810
:203BC00053F82430DB6803B198470134F2E72B6800221A7338BD00BF7C120020005C004022
:203BE0003806002000E100E0440B0020B80C0020034B1B6D03EBC00043000248184470472F
:203C0000005C0040046000408B4B2DE9F74F1B688A4C0025C0229D725A722565226848F6A5
:203C20008F13134043F40073284623601021FFF759FE226D824B5200134480221A60236DC5
:203C400040215B0003F1804303F5C0431960226848F68F6313402360284602F089FB23687E
:203C6000012523F4804323F0700343F4004343F0800383F440532360AC0004F1804404F5A3
:203C8000B8442368E8B223F4804323F0700343F4004343F0800323602368590406D52268A3
:203CA00048F68F73134043F4804323600021FFF719FE23685A0606D5226848F68F731340E3
:203CC00043F0400323600135082DD5D14FF000085C4B00201B68984580F0A1804FEA880B0F
:203CE0000746594B1B6853F80B305A78974280F090809B6A0C2404FB0734A67AE17AB50000
:203D000005F1804505F5B8452A6848F68F1313404E4A01F0030132F81120DFF820A1134356
:203D20002B60E37A296813F0040F48F68F630CBF00224FF480720B4013432B6063684FEA72
:203D4000C60903F14043A3F5C0434FEAA30CE37A4FEA4C0C1FFA8CFC13F0080FDAF85020AF
:203D60002CF0010337D04A44520002F1804202F5C0421360304620218DE80810FFF7B2FD32
:203D80009DE80810E27A12F0040F40D0DAF8502025894A44520002F1804202F5C042136014
:203DA000DAF8503009F104026D081A4452000CEB050302F180429BB202F5C04223F001037B
:203DC00013603046FFF714FF218905604908304602F0CEFA1BE009F104094A44520002F18C
:203DE000804202F5C0421360E37A5B0703D43046218902F0BDFA2B6823F4804323F0700343
:203E000043F4004343F0800383F440532B60013767E71B6903B1984708F1010858E70C4BA8
:203E2000012218800B4B18800B4B1B681A7303B0BDE8F04F02F078BE7C120020005C00406A
:203E400008600040440B0020B80C0020740100204A0B0020E00C0020380600202DE9F04F9E
:203E6000884B91B01860884B01221960874B08911A700023864A87495A5087495A50043334
:203E80001C2BF7D10024C0210491A146A346A24608998C4200F0AA807A4B1B6853F8245031
:203EA00003EB840205932B7809920A93AB8885F802A04B44C82B01DD0020E0E0734B4FF08C
:203EC00000081878AB6A0A336A7890457FD20C2202FB08F20B925A78A3F10A06920644BF1D
:203EE0000BF10100C0B206960246072A6CD8099F0B9E3F68B96A07970E440D9600214FEAF2
:203F0000810CCDF830C00026A1423AD2079F97F801C0664535D2DDF814C00C9F5CF8077083
:203F20004FF00C0CBF6A0CFB067797F80AC00E97944524D197F80BC00D9FCDF80CC0FF7AA1
:203F4000CCF3C00C0297C7F3C007BC4500F09480DDF808C01CF0100F40F08E80039F17F008
:203F6000100F40F0898007F0070CCDF838C0DDF808C00CF00707DDF838C0BC457CD1013629
:203F8000C2E7A14201D14645C5D30131A142B6D9049E069F710001F1804101F5C04143F85F
:203FA000061CFE7A5FFA82FC770733F8021C39D57C2931D8033121F00301049E314489B272
:203FC000B1F5007F049139D9304B187074E72F4BDDF828C018703148AB684844E2449847DB
:203FE000AB8801344B441FFA83F951E72C4A2D4B1168012019605168127A59601A7209F178
:20400000090292B283F804A05A80274B9A80274B0BF101021A7032E03707CBD43F3121F061
:204020003F01CAE73E2901D9360703D5013121F00101C2E71F3121F01F01BEE753F80A1CB4
:2040400011B9134943F80A1C069F1A70F97A53F80A6C11F0080F18BF0E4F4FFA8CF108BF9D
:204060000D4F01F1FF3C47F82C6008F101080C338B45B8BF934627E70132D2B235E711B0E9
:20408000BDE8F08FB80C0020440B0020400B0020BD6B0008BC0C0020240B0020590B002053
:2040A000489E0008500B0020200100203001002030B5039D144C08B1208104E06FF0500033
:2040C00020721E20607209B1618102E02420A072E1720E490E48002A08BF0A460D498A60E9
:2040E0000022934208BF03460B618A818A820A4B1DB903221A70257430BD8A8304221A7019
:20410000032323748D6130BD32010020789E0008429E00084801002068010020F8B5294B9B
:2041200003221C680C21204601F03EFA23684FF080521A61244B1B6823B1DB00013B1846C8
:204140000138FDD820460C21042201F02DFADFF8A8C01E4BBCF800201D4D1E4C1A800FCCBB
:204160000FC50FCC0FC594E80F001B4E85E80F000FCE1A4D0FC50FCE0FC5374657F820395E
:204180002B60174B174D1B88ACF80030A4F1200C0FCDACE80F000FCDACE80F0095E80F000C
:2041A00084E80F00104C0FCC0FC70FCC0FC723680E4933600E4B0F4A1868BDE8F84001F051
:2041C00091BD00BFD0A2000844010020480B0020480C002054060020A4060020240C002078
:2041E00030010020849E0008549E0008BC0C002038060020240B0020D0060020064B1860F6
:20420000064B00201980064B1A60064B064A1B689A615882FFF778BBD80C0020E00C002097
:204220004C0B00207C12002009390008034600201BB11A689B681044FAE770472DE9F84318
:204240001D4B80461C681D4B658A38B91868FFF7EDFF401B20824046BDE8F8831C6844B3E4
:204260000026334608EB050293421DD22068C0B11F18BD4216D29D428CBFC3EB05010021CB
:20428000BA429ABFC3EB0203C1EB0309C1EB000963680B48194430444A4604F0ABFC4E44FD
:2042A00000E01F46A46814B90548BDE8F8833B46D8E72046BDE8F8837C120020200B0020B4
:2042C000780C0020044B054A1860054B00201B689A615882FFF7B2BF200B00203D42000823
:2042E0007C120020064B1860064B00201980064B1A60064B064A1B689A615882FFF724BBA4
:20430000E40C00204A0B0020DC0C00207C120020493900080346998800680022FFF76EBFC1
:20432000F0B506461448B57A1C68006D776800EBC500124D400028580025C0F309008542BA
:2043400017D257F815601FFA86FCF6B20E550134B4FBF2F602FB16446E1C864209D24FEA81
:204360001C260E550134B4FBF2F602FB16440235E5E71C60F0BD00BF005C00400C60004042
:20438000F8B5069F06463D6807985B1BB3FBF2F402FB1434002CB8BFA41844B903785BB208
:2043A000002B02DCFF23037032E0047027E001230370338970689C42A8BF1C460023A342F8
:2043C0001CDA11F805E00135B5FBF2FC02FB1C5503F1010CA4455FFA8EFE02DBC0F800E073
:2043E0000CE011F805C001354EEA0C2E40F804EBB5FBF2FE02FB1E550233E0E73D60B07A61
:20440000FFF7F6FBA3B20360B07A3021FFF76AFA2046F8BD11220123834205D2013A02D00D
:204420005B009BB2F8E77047002B18BF18467047022830B54FF0000314BF002502250C2289
:204440005A43084CA018A2583AB1C27902F00202AA4202D182798A4203D00133082BEED11E
:20446000002030BDFC0D0020044A00231360044A1360044BFF221A70704700BFF80C0020CD
:20448000F00C0020EC0C002007B5074B074A1B680092074A0749019207484FF48072FFF7C6
:2044A0006FFF03B05DF804FBF80C0020F00C0020EC0C0020FC0C0020A801002010B502F087
:2044C0007F02212A044619469DF8080027D1012C19D0092C3FD1831E012B3CD8FFF7A8FFF9
:2044E0000446002837D0C379DB0702D4037A012B2FD02068A18804F1080289B2FFF7F2FED6
:204500000123237223E0032825D1FFF791FF034608B3027AFAB10068998889B214E0012A2A
:2045200019D1032C0ED0062C15D1222804D10B4B1868FFF7C7FE0AE021280CD10848FFF766
:20454000E9FE04E0074811460022FFF757FE002010BD032010BD022010BD00BFF40C0020D2
:20456000B8010020E80C0020114B10B50246044603F1180153F8040B8B4242F8040BF9D154
:204580001B7813700B4BA2789B781344A3700A4B227D9B7A13442375084B1868FFF746FE13
:2045A000074B20741B68C0F307206074E38210BDB89E00087C010020A8010020F40C0020CE
:2045C000B401002002F07F02212A05D10B2803D1024A00201360704702207047E80C0020E8
:2045E000431E402B034B28BF40201881024B1860704700BFA8010020B4010020014B186024
:20460000704700BFF40C002010B5022814BF0020022000230C225A43064901338C18E4798E
:2046200004F00204844204BF00248C50082BF1D110BD00BFFC0D002008B5054B00220220FC
:204640001A60FFF7E1FFBDE808400320FFF7DCBFE80C002070B50C4629B31449144A0B68D4
:2046600012680D469A1AD2B2C2F1FF02944201D9BAB11446002291B2A14202F1010205D2F7
:20468000465C0C49CE540133DBB2F4E72B600A4B1A781206FBD51B781B0604D5FFF7F4FE96
:2046A00001E0104670BD204670BD00BFF80C0020F00C0020FC0C0020EC0C0020A0F84110DB
:2046C00000F052BB026C6FF31722026400F04CBB90F84D300BB900F047BB704701230139A7
:2046E00003FA01F1D0F841300AB10B4301E023EA0103C0F84130FFF7EBBF40F2FF32914298
:2047000028BF114690F8452010B502F00F0201F00F0442EA041280F8452090F84620C1F3E1
:20472000051122F03F02114380F84610BDE81040FFF7CEBF10B540F2FF32914228BF11463D
:2047400090F8462001F0030402F03F0242EA8412C1F3870180F8462080F84710BDE81040A0
:20476000FFF7B6BF10B50021044606224B3004F04AFA002384F8493004F10800BDE81040B9
:2047800000F0F2BA38B503680446DB680D46984728B1236820461B6929469847012038BDB4
:2047A0000023137090F8613073B190F86030002B18BF013090F851309B0705D5A1F1610350
:2047C000192B18D82039C9B2080608D40D4B585C030616D50223137000F07F007047872969
:2047E00002D97831C8B270470123803903FA01F1002011707047A1F14103192BE4D82031B9
:20480000E1E77047F49E000813B50DF107020446FFF7C6FF18B99DF80700B0B921E00023B1
:20482000E21892F84B2082420FD00133062BF7D10023E21892F84B1011B982F84B0004E044
:204840000133062BF5D100200BE094F849309DF8072004F10800134384F8493000F084FAAB
:20486000012002B010BD13B50DF107020446FFF797FF68B10023E21892F84B10814203D141
:20488000002382F84B3006E00133062BF3D102E09DF8070060B194F849309DF8072004F1AC
:2048A000080023EA020384F8493000F05DFA012002B010BD38B50025044680F8435080F823
:2048C000445080F8455080F8401080F8421000F04BFA84F8405084F8425084F8435084F8CB
:2048E000445084F845502046BDE8384000F03CBA30B590F8405080F8431080F8425080F860
:20490000442080F84530BDE8304000F02DBA90F840208A420CD0002280F8401080F8421016
:2049200080F8432080F8442080F8452000F01CBA704790F840301943FFF7E9BF90F840307C
:2049400023EA0101FFF7E3BF002202604260826080F874208281C28102677047016070471E
:204960004160704781607047F7B590F8745004460DBB06462F46236F9F4205D2B36ABBB1A9
:20498000B06D9847A0B916E0A368A089E189009394E80C00FFF78CFB04F11000216FFFF70B
:2049A0005DFA40B10125FFF7B9FB84F8745002E001370436DFE7284603B0F0BD002303672A
:2049C000704770B5056F0024AC420AD005F1160650F82660964207D100EB840636698E4227
:2049E00002D1052C02D90DE00134EDE700EB8406B362049BAC4231613364B26504D301357E
:204A0000056701E0002070BD012070BD0148FFF79BBF00BF5C0E002010B50849044601204B
:204A2000FEF7A0FE06490220FEF79CFE6069FEF77DFEA069FEF786FE012010BDD54A000813
:204A4000854A0008FEF7D0BE07B501210DF10700FEF7D6FE01280CBF9DF807004FF0FF3052
:204A600003B05DF804FB07B501210DF10700FEF7E3FE10B19DF8070001E04FF0FF3003B017
:204A80005DF804FB10B50B78222B20D1104CFEF71BFF2378032B0DD8DFE803F00702070752
:204AA00000280CBF0223012303E000280CBF032301232370FEF710FFB0F5966F07D12378E6
:204AC000022B04D100200A2100F0B8FDFEE710BDD40E00201D4B73B51A78022A34D10322B8
:204AE0001A70FEF781FE03282ED9FEF77DFE0422011F01A8FEF7CAFE9DF80430312B23D151
:204B00009DF80530452B1FD19DF80630412B1BD19DF80730462B17D10D4C4FF0C2466FF024
:204B2000060544F001040B4B184685464FF001002146324604B402B401B401B401B401B451
:204B400001B401B4AE46704702B070BDD40E0020594B00080008002008B500F0CCFB00F027
:204B6000D7FB0A2044F24C2100F0DEFB00F0D6FB034B18460138FDD8BDE8084000F09ABD1E
:204B8000FF340C0007B50023024600930349044B0448FFF716FF03B05DF804FB30000020D3
:204BA000194A00085C0E002070B50E4615460024AC4205D23019291BFEF73EFE0444F7E75F
:204BC000204670BD13B50446FEF70EFE30B120460DF107010122FFF7E7FFF5E702B010BD88
:204BE00008B5064B1B681B7B052B05D1FEF76CFE003018BF012008BD002008BD38060020F9
:204C000070B50E461546FFF7EBFF48B146B10024AC4205D23019291BFEF7B2FD0444F7E7B0
:204C2000002070BD07B502AB03F8011D19460122FFF7E6FF002003B05DF804FB38B50546E9
:204C400008460C4604F0B4F8214602462846FFF7D7FF002038BD10B504464068FFF7C0FCAD
:204C60002269A3693AB9802213E05A791A710AB119680A709B6B002BF7D104F10C0010E017
:204C8000997949B159791971197909B1186801709B6B002BF4D103E0511C1A71CAB2F3E748
:204CA000A068FFF7ABFC012010BD000007B50023024600930349044B0448FFF782FE03B097
:204CC0005DF804FB7C010020574C00085C0E00200AB9037843B300238B63836923B98161BF
:204CE00006E09A6B1AB113468B42FAD11CE0996382681AB901F11403836006E093680BB1CF
:204D00001A46FBE701F11403936001F120029A6001F12C038B62002381F8343081F835305B
:204D200081F8363081F83730704700002DE9F041457804460E46174698468DB90948FFF793
:204D40003DFEC4F80C80276165612046FFF7AEFF3046FFF717FFBDE8F0410248FFF704BE1F
:204D6000BDE8F0815C0E002038B50489056834B128462146FFF76EFC241A0544F7E72046C7
:204D80002146BDE83840FFF765BC0346F0B5DD6800200A4698615861586218621863D8623A
:204DA00055B398791E8A4FF0FF34A8B9B04211D2611C11D12F5C852F04D1441CB44228BFDA
:204DC0004FF0FF3407F00307032F16BF01300530C019EBE70121997199799D6109B15E6193
:204DE0000AE0191D596201215C6119626118E4430D4426441D63DE62D86B1946BDE8F040EC
:204E0000FFF766BFF8B5069E04469DF81C509DF82070C16322B11168C1605168016101E029
:204E2000C260028225B901332360731E238101E02360268120680021228903F0E4FE6571F8
:204E40002EB125B11FB923681D70A77101E00123A37120460021FFF798FF2046F8BD00004D
:204E600013B5114C0322D4F8C00094F8CC1000F09BFB94F8CC204FF4803101FA02F2D4F847
:204E8000C00003681A6100230193019BB3F5007F02D2019B0133F7E794F8CC10042200F0F2
:204EA00083FB02B010BD00BFC09F000801498D460149084700500020BD4E000808B5124B7C
:204EC000124A1968914201D0002301E0104B07E01048D4188442F9D2C858D0500433F7E7E1
:204EE0000D4A934203D2002243F8042BF8E703F053FE00200146024602F060F8074B0BB1FB
:204F000003F036FEFEE700BF74A4000800000020380700203807002088120020718B00080A
:204F200008B50D4B1A680AB90C4A1A601B680C4AD21A824204DB09494242591A914206DAE3
:204F400003F010FE0C2303604FF0FF3008BD024A18441060184608BDD80E00208812002090
:204F600088EB0028FEE702F043B800000B4B10B5196809220A230A4801F064FF094B0222B2
:204F800019680948032301F05DFFBDE81040074B074819681A321B2301F054BF7004002093
:204FA000DC0E002074040020F40E0020780400200C0F002010B5044600F082F9034B204628
:204FC0001978BDE8104000F017B900BFB4020020F8B50446056800F0A7FC22680023510100
:204FE00001F184410B60802129600121A9622B61EB606379696113B18B4203D02BE04FF409
:2050000000436B644FF6FF73D36200256E1CF7B22046394600F092FCD0B1236848F6FF711D
:2050200003F1340242F8251018336D1017F0010F53F8252014BF6FF0FF016FF47F4101EA28
:20504000020214BF68214FF4D0410A4343F82520042E3546DAD1216801224B01490103F141
:20506000844301F18441C3F880220A60F8BD000038B5274B274C1A68012042F010021A6003
:2050800000F070FA0025002000F038FB65602368182023F40023236000F03DFB102000F0C1
:2050A0003AFB00F043F8A560102000F027FB102000F03FFB0028FAD000F039F8164800F08E
:2050C00045FB182000F01AFB182000F032FB0028FAD0022000F002FB0021104800F0D2FAC8
:2050E0004BF67F3000F098FB00F039F80C4B188800F0D4F80B4800F0D5F80B4800F000FC1A
:20510000FFF7AEFE00F02DF8FFF72DFF38BD00BF0020024000100240B8020020002000084C
:20512000B6020020B54F0008D14F0008704708B50020014600F048FB01204FF4806100F020
:2051400043FB0021022000F03FFB2D2000F04CFBBDE8084003204FF4800100F035BB00F07C
:205160000BBA00F049BA00000000000000000000012007E0022005E0032003E0042001E05D
:205180000520FFE70D4A0121116072B60C4A00211160074902B4084902B486B005498E46A5
:2051A000704700BFAFF30080AFF30080AFF3008000000061F9FFFFFF6D6D000814ED00E0F9
:2051C00010E000E0AFF30080AFF30080AFF30080FEE710B50446007900F0C4FA2079BDE840
:2051E000104000F0D7BA03689A6822F4602242F48012114399607047002370B51A461C4603
:20520000072B4FEA430503DCEE1801FA06F634431D4401FA05F501330A2B42EA0502EFD1D6
:205220000368DC601A6170BD38B5124D2A6813681C68A10706D5196821F0020119609368B6
:2052400003B19847620708D52B681A681B69116821F00401116003B19847E30708D52B68EF
:205260001A68DB68116821F00101116003B1984738BD00BFE4020020036801225B0103F141
:20528000844303F58673191F1A6018680028FCD143F8042C0B68002BFCD170470146042037
:2052A00000F092BA044B10B504461868A047034B1868A04710BD00BFE4020020E0020020A4
:2052C00010B50446FFF785FF20464FF46021FFF78AFF2368012103F1404308335A015B0186
:2052E00002F1844203F18443116520461960BDE81040FFF7C1BF08B5142000F033FA042048
:2053000000F030FABDE80840042000F043BA0000014B01221A60704720000E42014B0022F7
:205320001A60704720000E42431E092B06D8800000F1804000F5D84000B10160704738B565
:2053400050F8313004464D1E03B19847AA00012101FA02F223685A6038BD0000024B0121F8
:205360001868FFF7ECBF00BF28030020024B02211868FFF7E4BF00BF28030020024B0321FE
:205380001868FFF7DCBF00BF28030020024B04211868FFF7D4BF00BF28030020024B0521FA
:2053A0001868FFF7CCBF00BF28030020024B06211868FFF7C4BF00BF28030020024B0721F6
:2053C0001868FFF7BCBF00BF2803002038B50446274D9DF8100045F83420012805EBC4050F
:2053E0006B6004F5022512D00AD3022814D1AB0003F184430122C3F80021C3F880210BE048
:20540000AB0003F184430122C3F8002104E0AB0003F18443C3F880012046AD0000F096F810
:2054200005F1844501232B600F2C1FD8DFE804F0080A0C0F1215151515151A1A1A1A1A1ACD
:2054400040220CE080220AE04FF4807207E04FF4007204E04FF4806201E04FF40002054B22
:205460001A6038BD034B4FF480725A6038BD00BF240F002000E100E007B500930023FFF750
:20548000A5FF03B05DF804FB01F0030189000F238B408A4010B5046824EA0303134303601E
:2054A00010BD0000084A10B552F83030044653B102EBC00250689847012303FA04F4034B63
:2054C0005C6100BF00BF10BD240F002000040140104B2DE9F047104DD3F8149004468A469E
:2054E00005EBC0050026984654450CD80127A74017EA090F04D02B6813B1686898473E43F3
:2055000001340835F0E7C8F8146000BF00BFBDE8F08700BF00040140240F00200020FFF707
:20552000C1BF0120FFF7BEBF0220FFF7BBBF0320FFF7B8BF0420FFF7B5BF05200921FFF762
:20554000C7BF0A200F21FFF7C3BF000003460A4600F0FC01024808441946FFF795BF00BF6F
:2055600008000140034B1A6822F0070210431860704700BF0020024008B5074801F071FEE8
:20558000064801F06EFE064801F06BFEBDE80840044801F066BE00BF2C0300203403002005
:2055A0003C0300204403002070B501F00704A4000F25A5400368C80853F82060092A26EAFE
:2055C000050514BF1646082606FA04F4082A44EA050443F8204006D1012000FA01F1DA6842
:2055E00022EA010106E0092A05D1012000FA01F1DA681143D96070BD08B5032000F0B2F82B
:20560000BDE80840032000F0C5B80000014801F039BE00BF4C030020014801F033BE00BFC4
:2056200084030020014802F019B800BF4C030020014802F013B800BF84030020064B45F295
:2056400055521A604CF6CC42586099601A604AF6AA221A60704700BF0030004000284FEAE1
:20566000011105DA064B00F00F00C9B21954704700F16040C9B200F5614080F80013704766
:2056800014ED00E021F0604138B521F07F01084B0843986000241D4660B20F210134FFF76F
:2056A000DDFF2B2CF8D1F02385F8233038BD00BF00ED00E0044A054BD16801F4E0610B432F
:2056C000D360BFF34F8FFEE700ED00E00400FA05014B13F810007047D8A20008064B5A689F
:2056E00022F0030202435A6080005A6802F00C028242FAD1704700BF00100240030A0121CC
:20570000C0B201FA00F003F1804303F504331A68104318607047030A0121C0B201FA00F0B6
:2057200003F1804303F504331A6822EA000018607047030A0222C0B202FA00F003F1804380
:2057400003F504331B68184070470000044B05C85968126821F4741102430A435A60704794
:205760000010024010B50446FFF7B2FF074B53F82020074B03EB4404637803EBC2039B0093
:2057800003F1844301221A6010BD00BFBC030020D8A2000810B50446FFF79AFF084B53F888
:2057A0002020084B03EB4404637803EBC2039B0003F1844301221A6000221A6010BD00BF77
:2057C000C8030020D8A2000810B5054B054C5A6854F8200022EA00021143596010BD00BF21
:2057E0000010024034A3000810B50446FFF770FF074B53F82020074B03EB4404637803EBD6
:20580000C2039B0003F1844300221A6010BD00BFD0030020D8A20008024B072258601A6028
:20582000704700BF10E000E008B5044B1A6801321A60034B1B6803B1984708BD4412002048
:20584000A40F002011F0010F70B542EA03030CBF0825002503FA05F5006801F1FF3400F17B
:205860001800C4F3400450F8241014BF6FF0FF066FF47F463140294340F8241070BDF8B517
:2058800007680546FB683E691E4016F0400403D0046A0CB1A0474024F30604D5AB6913B1A9
:2058A000984744F01004300704D56B6913B1984744F00804710704D52B6913B1984744F03E
:2058C0000404B20704D5EB6813B1984744F00204F30704D5AB6813B1984744F00104E44315
:2058E0003C61F8BD0368013903F140432033DB0003EB8101890001F1844101230B60704716
:2059000010B504460448A0470448A0470448A0470448A04710BD00BF240400204C04002068
:20592000DC0300200004002010B504460079FFF719FF2079BDE81040FFF72CBF03791E2B7A
:2059400010D9212B0ED0202B0ED9222B01D0252B04D102298CBF0020012070474B1E58424E
:205960005841704701207047002070470368002203F140430C3301EBC3039B0003F18443DD
:2059800002311A6040F82120704738B505460C4613460022FFF756FF28462146BDE83840E8
:2059A000FFF7A0BF38B543790446022B0D463ED0042A3CD8DFE802F00312202A3600FFF78B
:2059C000D5FF2368013D03F140432033DB0003EB85039B0003F18443002221E00368002209
:2059E00003F140430C3301EBC3039B0003F184431A606022082301E010220023FFF722FF75
:205A000020462946BDE83840FFF76CBF03684FF2F1129A6103229A605B0103F18443012270
:205A20001A6038BD0122BDE83840FFF7AEBF38BD10B5074B1C68E16822690A40120605D5B4
:205A40005B6A1BB198476FF08003236110BD00BF2404002010B5074B1C68E16822690A40E3
:205A6000D20705D59B681BB198476FF00103236110BD00BF24040020F8B50B4F3D68EB680B
:205A80002E691E4016F0400403D03C6A0CB1A0474024B30604D5FB6913B1984744F0200455
:205AA000E4432C61F8BD00BF24040020F8B5124E3768FB683D691D4015F0100403D0B4695B
:205AC0000CB1A0471024290704D5736913B1984744F008046A0704D5336913B1984744F069
:205AE0000404AB0704D5F36813B1984744F00204E4433C61F8BD00BF240400200148FFF71C
:205B0000BEBE00BF4C0400200148FFF7B8BE00BFDC0300200148FFF7B2BE00BF00040020D5
:205B2000D36870B59B0638D513689E0635D513689D0702D41368DC0701D553682DE0556880
:205B4000C4888388A4B201349BB29C42EDB2046808D0C6880389B6B29BB29E420FD18388FB
:205B60009BB263B983889BB2E35C86880389B6B29BB29E4235D0838801339BB28380C38817
:205B80009BB2E554C4880389A4B29BB29C4217BFC388002301339BB2C380D368180622D5CE
:205BA00013681B061FD58888CB8880B29BB2984212D088880B6880B2185C8C880B89A4B290
:205BC0009BB29C4218BF8B88C0B21ABF01339BB200238B80506070BDD36823F08003D360D5
:205BE00070BD0023CAE770BD02480349034AFFF797BF00BFB40F0020A80F00200038014056
:205C000002480349034AFFF78BBF00BFC00F0020D80F00200044004002480349034AFFF74F
:205C20007FBF00BFCC0F0020E40F002000480040294B072818BF18701A78052A49D8DFE826
:205C400002F003131E222A35244A4FF6FB71106C014011644FF43F41116406221A70204BF7
:205C60001B685A7B1A7370471C4A4FF6FB71106C014011644FF43F41116404222AE00222B3
:205C80005A70032226E05A78013AD2B25A705B780BBB04221BE0114A116C89B241F01001A5
:205CA000116405221A700A225A7070475A78013AD2B25A705B7873B9084A4FF6EF73116C41
:205CC0000B401364064B1B685A7B1A730622024B00E006221A7070474C120020005C0040F4
:205CE0003806002070B50446807B0D461646FFF739FD084A084B09491A60094B09480B6080
:205D00000949656008600221A6601B681172984770BD00BF5C1200207C1200205412002048
:205D200054060020A406002078120020F8B56C4D6C4B2A685C6C1268A4B202F480622242F2
:205D400006D06FF480625A64674B1B685B6898472B681B6823409F0403D5624A6FF400513F
:205D60005164DE0406D55F4B6FF4C0525A640020FFF75EFF2A681168214008050FD5594B60
:205D8000186C80B240F0080640F00C001E641864107B5073032010736FF4C0525A648B051E
:205DA00003D5504B6FF400725A64CF0506D54D4B6FF480725A640720FFF73AFF2B681B6817
:205DC00003F40043234200F08980464B5A6C110440F184806FF4004112F00F06596458D1E9
:205DE000196848F6800008400028EED088B23F4C00F4405525803E4D00F030002880186870
:205E0000D60620F4804020F0700040F4004040F0800080F400501860186820F4E04020F02E
:205E2000400040F4004040F0800080F02000186001D5080607D5196848F60F720A401A6032
:205E400000F08EFE0BE0186840F68F7202401A600A0502D500F09CFC01E000F001FE214BBE
:205E600022881968288821F4804121F0700141F4004141F08001514019601A6822F4E04203
:205E800022F0400242F4004242F0800242401A60F8BDB40004F1804404F5B84427683B04A1
:205EA0000CD5226840F68F7313402A682360926806F18043013B52F823309847380684D5D4
:205EC000226848F60F73134023602B6806F180465B68013E53F82630984776E7F8BD00BFFF
:205EE00038060020005C004054120020481200204A120020800000F1804000F5B8400368A3
:205F000023F4804323F0700343F4004343F08003594001607047000018B9034B07221B6875
:205F20001A820248704700BF7C1200209C06002037B5114B1A681D46127802F07F02212A20
:205F400001D0022016E0A0F12003012B0B4B0C4C1B6888BF002423B102A901F8010D022034
:205F60009847002CEDD02B68002528469C615D82A047284603B030BD7C1200200012002082
:205F8000195F000813B5104B1B681A7802F07F02212A14D1022806D0222806D19A780B4B1D
:205FA00002F003021A70002400E00224084B1B6833B102A901F8010D0220984700E00224C3
:205FC000204602B010BD00BF7C120020F00F00200012002021B9022834BF0020022070472E
:205FE00002207047044B1B689B7A1BB1034B05221B681A73704700BF7C120020380600200E
:20600000024B04221B681A73704700BF38060020054B1B689B78032B04D8044901EBC3013C
:2060200000F088BB002070477C12002084060020014900F07FBB00BF4C060020014900F01F
:2060400079BB00BFC80600200C4B00221B6801219A720B4B4FF4E05019640A4909681A64AD
:206060005A6418644FF43F405A6408601864064B4FF4801018600A73704700BF7C12002045
:20608000005C00403806002000E100E02049214B0A681B6870B59B1A13F0FF030E461E49E1
:2060A00005D10A78013AD2B20A70FAB170BD0120087000211948402B28BF40230C46184DF0
:2060C00011F0010FAD5C01F10101EDB21CBF44EA0525056002F101020CBF2C460430994239
:2060E000D2B2ECD3D90748BF046032600D4A0E49106D40000B50536823F4E04323F040036F
:2061000043F4004343F0800383F03003536070BD08120020F4100020F81100208061004021
:20612000F10F0020005C0040146000402DE9F843494B4A4C1B6800254FF0C0089D7283F83B
:2061400009802565236848F68F16334043F400732360236848F2800723F4E04323F0400342
:206160003B4383F010032360226D3D4B52004FF0400943F80290236D80225B0003F1804396
:2061800003F5C0431A602368284623F4E24323F070031B041B0C2360324B1B6893F82C103F
:2061A00000F0E6F828464FF44051FFF7A3FEA3680220334043F4C063A360226D2A4B5200E5
:2061C00013444FF480721A60A368294623F4E04323F040033B4383F02003A360FFF78AFE1A
:2061E000E36803203340E360226D204B520013444FF488721A60494600F0BAF803204FF48A
:206200004051FFF777FE636801201E406660226D174B520043F802806368294623F4E043FE
:2062200023F040033B4383F020036360FFF762FE104B01221B6828461A7300F075FC0E4B25
:20624000FF221D600D4B1D600D4B1D600D4B1D600D4B1A70BDE8F8837C120020005C0040D5
:2062600008600040541200202060004038600040106000403806002004120020FC110020E7
:20628000F410002008120020F811002070B50C4611B31249124A0B6812680D469A1AD2B20D
:2062A000C2F1FF02944201D9A2B11446002291B2A14202F1010205D2465C0A49CE5401336D
:2062C000DBB2F4E72B60084B1B781B0604D5FFF7DDFE01E0104670BD204670BDF4100020FF
:2062E00008120020F10F0020F8110020034B1868034B1B68C01AC0B2704700BF0412002084
:20630000FC1100200A4B10B51A680A4B1B689B1ADBB2994228BF194600238B4206D0064C61
:20632000A45C0132C454D2B20133F6E7184610BDFC11002004120020F810002010B5FFF70C
:20634000E1FF094A044613680344DBB21360074A1268D31ADBB2402B04D803204FF440517B
:20636000FFF7C8FD204610BDFC11002004120020104B3E291B6D03EBC0000F4B4FEA400001
:2063800003440ED94A09C80608BF02F1FF32C1F3090108BF92B241F4004141EA82221A603B
:2063A00070474A08C80748BF013241EA82211960704700BF005C00400C60004010B5064CAF
:2063C00018B9236801221A8210BD044B1B681B68984720680A3010BD7C12002078120020BA
:2063E00010B5064C18B9236801221A8210BD044B1B689B68984720680C3010BD7C120020AB
:206400007812002010B5204B18B91B6802221A8210BD1E4A1968002010800C78134614F047
:206420007F040DD14A7A910644BF0221197012F0400F1A7814BF22F0010242F0010214E0FD
:20644000012C1FD0022C1ED1097901F00F02920002F1804202F5B84211F0800F126806D067
:2064600002F03002102A07D101221A7004E002F44052B2F5805FF6E7054B1B681B69984734
:20648000024810BD104610BD7C1200204E12002078120020234A2DE9F84314689046238A2D
:2064A000267A214FA3B9042E12D120490A78012A0AD11F4A10681F4A80B2024452001360E3
:2064C00030223A800B7027E010233B80072623E0A58AAB428CBF022604269D4228BF1D462E
:2064E0002846A36998478146002000F0CFFB2A460146484600F063FB2946002000F0E2FBB3
:20650000238A4FF440525B1B2382638A1D4430233B80094B65821A80D8F800301E72BDE878
:20652000F88300BF7C1200204A1200200C120020505C0040023000204812002010B50A4BE7
:206540000A491B6849789A7891420AD3D97841B99C8834B99A72064B1B685B68984720469E
:2065600010BD022010BD00BF7C120020D00600207812002038B50E4A0E4C126823689269B3
:2065800018799978904723689A7A7AB170B95A7962B9DD7855B9084B1B68DB6898472368BB
:2065A00028461A79DA729A781A7338BD022038BD541200207C1200207812002038B52F4B9E
:2065C0001B68187810F07F0004D15A7A22F020025A7238BD02284ED15A88002A4CD15A7946
:2065E000002A49D11A79264D22F08000840004F1804101F5B84109682D7812F0800F14BF1C
:2066000001F0300101F44051A84234D2002932D09B7A83B304F1804404F5B844120623681B
:206620000CD503F03003102B1FD1C4B2204600F01CFB2046302100F0F3FA16E003F4405331
:20664000B3F5805F11D128B90E4B93F82C1000F047FB01E000F0F9FA236823F4804323F062
:2066600070039BB283F440532360074B1B685B699847002038BD022038BD00BF7C120020BC
:20668000D0060020540600207812002038B51D4B1D4D19682D780A7922F08004A30003F14B
:2066A000804000F5B840006812F0800F14BF00F0300000F44050AC4222D24C8804BBF8B19F
:2066C000897AE9B103F1804303F5B84312F0800F1A6807D022F4E04222F0400292B282F047
:2066E000100206E022F4804222F0700292B282F480521A60054B1B689B699847002038BD75
:20670000022038BD7C120020D00600207812002008B5064B1B685A7A42F020025A72044B40
:206720001B68DB699847002008BD00BF7C12002078120020054B1A68538A18B98988CB1A41
:206740001382704708681844704700BF7C12002008B50B4B002093F82C1000F0C1FA094B04
:206760001B68187A082806D1074B4FF480521A80064B10221A80B0F109035842584108BD3A
:20678000540600207C120020481200204A12002073B5934E934B3268934D92B213445B0084
:2067A0001A682B68197A09290FD092B2520002F1804202F5C042117819705178597091881F
:2067C0005980118999809289DA8001221A72DA885C78002A61D11A7812F07F023AD1092C22
:2067E00002D1FFF7ABFE44E0052C0FD193F90220002A01DA08234DE0DA78002AFAD19A887E
:20680000002AF7D19B7A002B37D0F3E7032C13D19A78012A07D0754B20461B685B699847F2
:20682000032828D135E09A88002AF4D15B7A9806F1D5FFF76DFF1CE0012CECD19A78012A50
:20684000E9D19A88002AE6D15B7A9906E3D5FFF7B5FE0EE0012A04D10B2CDCD1FFF78AFE56
:2068600007E0022AD7D1012CF1D0032CD3D1FFF70DFF10B1CFE70028BCD132685C4B92B2E9
:2068800013445B0000221A605A4B30221A80062300E009232A681372CEE0062C13D11A7877
:2068A000520677D1DA78514B012A02D11B68DB6967E0022A02D11B681B6A62E0032A69D18E
:2068C0001B685B6A5DE0002C3CD15988002961D15A6822F0FF02B2F5003F5BD11A7812F043
:2068E0007F0204D19B88002B00F0AA8052E0012A0CD13E4A1879126892699047002849D1F9
:206900002B689B7A002B40F09B8043E0022A41D11B79394803F00F018A0002F1804202F5AA
:20692000B8421268007813F0800F14BF02F0300202F4405281422DD213F0700F2AD1002AF1
:206940007ED127E0082C03D11B785B067AD021E00A2C1FD11A7802F07F02012A1AD19A7A45
:20696000C2B15988B1B95A6822F0FF02B2F5803F10D11E4A1879126892699047002863D09D
:2069800008E03BB12A680024548293612046984720460AE0154B1A682B6812695878904777
:2069A000032802D1104B1B6805E02B684FF6FF711A8A8A4201D1092203E0022800D012B9B9
:2069C00008221A7238E093F9001000292EDAD988019101988242054810D9019A1A821EE061
:2069E000505C0040043000207C12002054120020023000204A120020D00600208A420ED2B3
:206A0000016891F82C108A4201D2002105E092FBF1F401FB142212B901210C4A11700268D1
:206A200092F82C209A82FFF735FD05E003221A72074B4FF440521A80FFF78AFE02B070BD88
:206A4000044B9FE7044B9DE7044B9BE70C1200204812002005640008BD630008E163000820
:206A6000F8B52B4D2C68237A032B01D0052B41D1A369228AABB1A2B1A68A964228BF1646CD
:206A800030469847238A07469B1B2382638A00203344638200F008F932460146384600F0C5
:206AA000A6F8238A53B11B4B00204FF4405201461A8000F007F9184B30221A80238AA28A33
:206AC0009A4202D82B68032202E01BB12B6805221A720CE02A6806211172104A1168104AFF
:206AE00089B20A44520013600B4B30221A802B681B7A06E0072B03D10A4B1B68DB689847F8
:206B000008232A681372BDE8F840FFF721BE00BF7C120020481200204A120020505C004032
:206B2000023000205412002030B50B4B1C780023A3420CD203F1805202F5B85291000D68FB
:206B400048F68F722A401A430A600133F0E7034B40F08000186030BDD00600204C5C004079
:206B600010B5134C23681A7A022A01D0042A04D1FFF790FC23681B7A13E0062A10D15A785A
:206B8000052A09D11A78520606D19878FFF7CCFF084B1B681B6A9847074B1B689B68984769
:206BA000082322681372BDE81040FFF7D1BD00BF7C1200207812002054120020704730B5E9
:206BC00001F10051013201F54051521049000023934200F1020009D010F8015C10F8024C8E
:206BE00044EA052421F823400133F1E730BD01F1005101F5405149005308F0B51C460E4600
:206C0000054634B156F8047B013C25F8027BA4B2F7E7D20744BF11F8232000F81320F0BD6C
:206C2000800000F1804000F5B8400368CA0623F4E04323F040039BB248BF83F010038A0601
:206C400048BF83F0200303607047800000F1804000F5B84003685B0406D5026848F68F7310
:206C6000134043F4804303607047800000F1804000F5B84003685B0606D5026848F68F733E
:206C8000134043F04003036070470000054B1B689BB203EBC00000F1005000F5405040003D
:206CA00000887047505C0040044B1B689BB203EBC000034B03445B0018887047505C0040A9
:206CC00004300020044B1B689BB203EBC000034B03445B0019607047505C00400230002035
:206CE0000D4B3E291B689BB203EBC0000B4B03444FEA430209D94B09C80604BF03F1FF334F
:206D00009BB29B0243F4004304E04B08C90748BF01339B0213607047505C004006300020C4
:206D200008B5114B01211C6803222046FEF73CFC002301211A469342206834BF02254FF47D
:206D40000035B2F5007F056103F1010303D0002A08BF012101E04FF0FF31B3F5007F04BF5A
:206D600052180023E7E700BFD4A2000808B5034B0BB1AFF3008062B6FFF7D2FF00000000B3
:206D8000C288838892B29BB2C188D31A828889B292B2914203D2028992B20132134498B203
:206DA000704710B5036904465868FFF7E9FF90B123695B6899881A6889B2505C99881A8925
:206DC00089B292B2914217BF9A880022013292B2C0B29A8010BD4FF0FF3010BD08B5036913
:206DE0005868FFF7CDFF08BD03695B689988DA8889B292B2914205D09A881B6892B2985C96
:206E0000C0B270474FF0FF30704703699A689088D18880B289B28842F9D11A6813685B06E6
:206E2000FCD5704713B504698DF8071020460DF10701012200F04CFC0028F7D0012002B070
:206E400010BD000030B5002545604FF47A758560024D016105600275437530BDC8A30008FA
:206E6000044B02791B789A4202D1034B1B681860704700BF2012002024120020002310B5B7
:206E80000446036072B6054B19311970044B18600448FEF735FD62B6204610BD2012002023
:206EA00024120020616E0008036801221B685B0103F184431A607047036801391B6889B2E9
:206EC0009962704738B5054639B9036801221B689962DA62D86A80B238BD30244C434FF6FD
:206EE000FF71B4FBF1F1013189B204EB5104B4FBF1F4FFF7E1FF2B68A4B21B682046DC6266
:206F000038BD000008B501210848FFF7B7FF02210748FFF7B3FF03210648FFF7AFFFBDE8CC
:206F2000084005480421FFF7A9BF00BF1012002014120020181200201C120020F8B5054662
:206F40000C4616468F18BC4206D02B6828461B6814F8011B9847F6E73046F8BD38B505463D
:206F60000C46084641B101F023FF2B6802469B6828462146984738BD38BDFEE7302830B5CE
:206F80000C4615D8A1B1012A04D0022A0CBF0223002300E01346074A000115181258287B5D
:206FA000117922460B39C9B2BDE83040FEF764BA30BD00BFC09F0008FEF75AB808B5FCF72E
:206FC00029F8FBF7CFFFFCE701F00CBE30280BD8064B03EB001043681A68437B343203F163
:206FE0008043013B42F82310704700BFC09F0008034B1A6822F0E06242F080621A607047DF
:2070000004000140302870B53BD8082939D8DFE801F0051A080B0E110814170000240322D4
:2070200013E00024042210E0002422460DE0002409220AE00024082207E001240B2204E006
:2070400001240F2201E0002407220E4B00011E18317B1858FEF7A8FA706890B1717B24B18F
:207060000122BDE87040FEF79DBC0368013903F140432033DB0003EB81039B0003F1844338
:207080001C6070BDC09F0008FFF730B907B501210DF10700FFF736F901280CBF9DF8070069
:2070A0004FF0FF3003B05DF804FB07B501210DF10700FFF743F910B19DF8070001E04FF0C9
:2070C000FF3003B05DF804FB002242604FF47A728260014A0260704708A4000870B516460C
:2070E0000D4631B10E4B1B681B7B052B03D0002070BD084670BD0B4B1B782BB9284631466C
:20710000BDE87040FFF7C2B80024B44205D22819311BFFF7BBF80444F7E7204670BD00BF0B
:20712000380600203812002007B502AB03F8011D19460122FFF7D2FF03B05DF804FB38B5C8
:20714000054608460C4601F033FE214602462846BDE83840FFF7C2BF70B50E461546002479
:20716000AC4205D23019291BFFF7E8F80444F7E7204670BD13B50446FFF7B8F830B120462F
:207180000DF107010122FFF7E7FFF5E702B010BD0148FFF799BF00BF2812002030280ED8A1
:2071A000084B00011A18127B012101FA02F21B581B689B681A420CBF002001207047002073
:2071C000704700BFC09F0008302810D8084B00011A18127B1B58012000FA02F2D1F1010139
:2071E00038BF0021090102FA01F11B6819617047C09F00080A4B1A680A4B9B6800BF00BFB7
:20720000074909688A42F5D1C3F53B4330218033B3FBF1F34FF47A7000FB0230704700BF7F
:207220004412002010E000E038B50446FFF7E2FF054644B100F014F8FFF7DCFF401BB0F5ED
:207240007A7F01D2F5E738BD013C05F57A75F3D138BD20B1C000431E18460138FDD870479D
:20726000704710B504460079FEF77CFA2079BDE81040FEF78FBA03685A6822EA01015960A4
:2072800070470000F0B5036885B01A68002501925A69044602928B4A03951268C260426A62
:2072A000960600F1C6804268002A00F0D58151889588C8077ED50299C90704D51288520099
:2072C00042F0010280E002998F072AD5012D019A0EDC22F4806201921A609A690392019AFE
:2072E00042F4007201921A60002D00F0928113E0022D0BD142F4006201921A609A6903926E
:20730000019A22F4806201921A6005E042F4806201921A609A6903925A6842F480625A6097
:207320009AE1029802994606C1F380011AD5E1B9032D01DC012D09D1D1881B6990684E1C3F
:20734000D68043549388013B938007E0AB1E012B04D820464FF48061FFF78DFF012D00F3F1
:207360007B8156E1002900F07781032D03D1019921F4806104E0022D04D1019941F400710D
:2073800001911960D1881B6990684E1CD68043549388022D03F1FF33938040F05D81D388CA
:2073A0009168581CD08020680069C8549388013B93802EE10298C00708D51DB1596841F488
:2073C00080615960128852001A6145E10298870744BF986903900298029EC0F3C01076078D
:2073E00004D4D5F1010638BF002600E00126F6B218B9002E40F02C812EE175B1D1889668B4
:207400004F1CD780715C013D19619580002800F02381002D40F02081A3E0002E00F01C8118
:207420004A0700F1F680019A42F4007201921A60EFE0029A970747D59A6985600392039A05
:20744000D60619D4039A12F0800F9A680CD0100408D59A68DD6840F2013305F0FE0513406E
:207460001D4309E0DD6805E011049D6802D5C5F3090501E0C5F34605039B606B13F004038B
:2074800014D038B1C3882BB1E36A03B19847636B0022DA80206B60B1A36A0022058082807C
:2074A000154603B19847236BDD8002E008B10580C38023685A6842F480625A60032384F8CF
:2074C0002330C9E044120020029AD20615D59B69406B039338B1C3882BB1E36A03B19847A7
:2074E000636B0022DA8023681968019A42F4806201920A431A600123E1E70298029DC0F351
:20750000800015F0800518BF5D689A6918BFC5F380250392039A12F0040228D0226B1AB104
:207520009688D188711A00E0114605F0FF0615B9002800F0918000208DF802003AB131B1AD
:20754000D0889568471CD7802A5C8DF802209DF80220D2B21A61002977D0002E7CD0012925
:207560007AD120464FF48061FFF785FE74E08DF80320029D626B15F040051CBF5D68C5F3B3
:207580008025EDB21AB19688D188711A00E011468DB190B90029E4DD1B699068DBB28DF8A4
:2075A0000330D388032903F10105D5809DF80320C25451DCD5E700284ED0032903D101982C
:2075C00020F4806004E0022904D1019840F40070019018601B690029DBB28DF8033006DDB8
:2075E000D38890685E1CD6809DF80320C254002D32D0236801291B69DBB28DF80330B0DD60
:20760000636BDA889968501CD8809DF803308B54A7E7A38B013B9BB2A3839BB120464FF46E
:207620008061FFF728FE636803F10C02DB89626013F0010F236814BF40F2015240F201121F
:207640001A6009E06360022339E7002E89D103E0002D7FF4D3AEE3E605B0F0BD13B50368D5
:2076600004465A6900929B690193184B1B68C360009B03F470638360436A99061CD54FF402
:207680008061FFF7F8FD23681A6842F480621A60009A520510D5606B6FF480625A6138B1F5
:2076A000C3882BB1E36A03B19847636B0022DA80012384F8233007E0236800225A619A613C
:2076C000FF2384F82330019B02B010BD44120020F0B583680546046800209F88DE88BFB2C3
:2076E000B6B2B74204D0E36823F08003E36027E026683606F7D59042F5D00E5C013066609C
:20770000EBE7DF889E88BFB2B6B20137B74211F800C01DD0DF881E89BFB2B6B2B74213D087
:20772000DF881E68BFB206F807C0DF881E89BFB2B6B2B74218D0DE880136B6B2DE800130CA
:207740009042AB68DDD303E09E88B6B2002EE7D19A88DB8892B29BB29A4200D1F0BDE36882
:2077600043F08003E360F0BD0026E7E72DE9F04120F00047FC0D7F3C162C064618DC002C5F
:2077800080461DDB194F2741074223D0184900F0F5FE002101F0B6F9E0B1002E04DD4FF437
:2077A000000343FA04F4A04428EA0700BDE8F081B7F1FF4F0ED3014600F0E0FEBDE8F0817C
:2077C0000B4900F0DBFE002101F09CF910B1002E07DB17B93046BDE8F0814FF07E50BDE806
:2077E000F0814FF00040BDE8F08100BFFFFF7F00CAF249712DE9F0478AB004460D4600F0BD
:207800009DF8DFF898A006469AF900300F4601330FD02046294600F0A5F950B14FF00008A2
:207820004FF0000942464B462046294600F008FE20B9304639460AB0BDE8F08716499AF887
:20784000006001220023CDE90445CDE9024501910092089366B9CDE90689684600F0AAF922
:2078600080B1089B9BB9DDE906010AB0BDE8F0874046494642464B4600F09AFC022ECDE9A3
:207880000601EAD101F06EF921230360E9E701F069F9089B0360E6E728A40008D206002065
:2078A00070B58AB0054600F009F9224C064694F90030013308D0284600F07EF920B1284695
:2078C000002101F001F910B930460AB070BD1A4901220023284601910092089300F0EAFACC
:2078E0002478CDE90401CDE902017CB900220023CDE90623684600F05DF988B1089BA3B9F3
:20790000DDE9060100F0E4FD0AB070BD0020002102460B4600F04CFC022CCDE90601E9D12B
:2079200001F020F921230360E8E701F01BF9089B0360E5E7D206002030A4000821F0004CBF
:207940002DE9F8434FEA1C5CDFF86C814FEA0C5CC44506460F460B46024600F08F80002955
:207960006FDD0F1578D0A7F2FF37C3F31303F90743F4801360D4D10F4FF0000C01EB430359
:207980007F105200654616204FF400116C189C424FEAD2764FEA420202DC1B1B65188C4410
:2079A000013806EB43034FEA5101EFD1804620264FF0004109E023D0D40F013E4FEA5101F7
:2079C00004EB43034FEA42021ED0AB4201EB0804F1DD04F00049B9F1004F04EB010809D04D
:2079E000A9465B1B944288BF03F1FF33121B08444D46E1E7B8F1000FF2DB05F10109F0E7AF
:207A00009442E6D91D46D7E71A4304D0431C41D000F00103184446084FEA6C031CF0010FAD
:207A200003F17F5303F5001318BF46F0004603EB07513046BDE8F883D10F01EB43035200E2
:207A400099E721F00043034322D051BB0F46D30A153F5205002BFAD013F480111DD15B005B
:207A6000D80201F10101FAD5C1F10100C1F1200422FA04F407448A40234374E702460B465D
:207A800000F06CFA32463B4600F0B6F8BDE8F883BDE8F8830CF1010CBEE720240120002184
:207AA000E6E702460B4600F0A5F802460B4600F07FFBBDE8F88300BF0000F07F20F0004230
:207AC000B2F1FF4FF8B5044603462DD25AB300283DDBB2F5000F4FEAE0502CD37F38C3F39E
:207AE0001603C20743F4000348BF5B00002740105B003E4619244FF08072B5189D4202DCBA
:207B00005B1BAE181744013C4FEA43034FEA5202F3D113B107F001031F447F1007F17C5745
:207B200007EBC050F8BDF8BD014600F02FFE214600F024FDF8BD14F400020FD15B001902E8
:207B400002F10102FAD5C2F101021044C6E7014600F012FD014600F0CDFEF8BD0122104435
:207B6000BCE700BF31F0004310B408D00F4AA3F5801494420AD804205DF8044B70470028BF
:207B80000CBF022003205DF8044B7047B3F5801F01D20320F7E7064A934201D00020F2E770
:207BA000D0F1010038BF0020EDE700BFFFFFDF7F0000F07F0020704730F0004001D1022063
:207BC0007047A0F50003B3F1FE4F01D204207047054B421E9A4201D803207047B0F1FF4395
:207BE00058425841704700BFFEFF7F0081F0004102E000BF83F0004330B54FEA41044FEABB
:207C0000430594EA050F08BF90EA020F1FBF54EA000C55EA020C7FEA645C7FEA655C00F080
:207C2000E2804FEA5454D4EB5555B8BF6D420CDD2C4480EA020281EA030382EA000083EA61
:207C4000010180EA020281EA0303362D88BF30BD11F0004F4FEA01314FF4801C4CEA11319A
:207C600002D0404261EB410113F0004F4FEA03334CEA133302D0524263EB430394EA050F59
:207C800000F0A780A4F10104D5F1200E0DDB02FA0EFC22FA05F2801841F1000103FA0EF276
:207CA000801843FA05F359410EE0A5F120050EF1200E012A03FA0EFC28BF4CF0020C43FAE7
:207CC00005F3C01851EBE37101F0004507D54FF0000EDCF1000C7EEB00006EEB0101B1F5A2
:207CE000801F1BD3B1F5001F0CD349085FEA30004FEA3C0C04F101044FEA445212F5800FA9
:207D000080F09A80BCF1004F08BF5FEA500C50F1000041EB045141EA050130BD5FEA4C0CF0
:207D2000404141EB010111F4801FA4F10104E9D191F0000F04BF01460020B1FA81F308BFFC
:207D40002033A3F10B03B3F120020CDA0C3208DD02F1140CC2F10C0201FA0CF021FA02F186
:207D60000CE002F11402D8BFC2F1200C01FA02F120FA0CFCDCBF41EA0C019040E41AA2BF86
:207D800001EB0451294330BD6FEA04041F3C1CDA0C340EDC04F11404C4F1200220FA04F07B
:207DA00001FA02F340EA030021FA04F345EA030130BDC4F10C04C4F1200220FA02F001FAD1
:207DC00004F340EA0300294630BD21FA04F0294630BD94F0000F83F4801306BF81F4801150
:207DE0000134013D4EE77FEA645C18BF7FEA655C29D094EA050F08BF90EA020F05D054EAC1
:207E0000000C04BF1946104630BD91EA030F1EBF0021002030BD5FEA545C05D140004941C0
:207E200028BF41F0004130BD14F580043CBF01F5801130BD01F0004545F0FE4141F47001B0
:207E40004FF0000030BD7FEA645C1ABF194610467FEA655C1CBF0B46024650EA013406BF6D
:207E600052EA033591EA030F41F4002130BD00BF90F0000F04BF0021704730B54FF48064C9
:207E800004F132044FF000054FF0000150E700BF90F0000F04BF0021704730B54FF4806407
:207EA00004F1320410F0004548BF40424FF000013EE700BF42004FEAE2014FEA31014FEAA3
:207EC00002701FBF12F07F4393F07F4F81F06051704792F0000F14BF93F07F4F704730B513
:207EE0004FF4607401F0004521F0004120E700BF50EA010208BF704730B54FF000050AE04F
:207F000050EA010208BF704730B511F0004502D5404261EB41014FF4806404F132045FEAF9
:207F2000915C3FF4DCAE4FF003025FEADC0C18BF03325FEADC0C18BF033202EBDC02C2F15B
:207F4000200300FA03FC20FA02F001FA03FE40EA0E0021FA02F11444C1E600BF70B54FF095
:207F6000FF0C4CF4E06C1CEA11541DBF1CEA135594EA0C0F95EA0C0F00F0DEF82C4481EAE1
:207F8000030621EA4C5123EA4C5350EA013518BF52EA033541F4801143F4801338D0A0FB96
:207FA00002CE4FF00005E1FB02E506F00042E0FB03E54FF00006E1FB03569CF0000F18BF03
:207FC0004EF0010EA4F1FF04B6F5007F64F5407404D25FEA4E0E6D4146EB060642EAC6210C
:207FE00041EA55514FEAC52040EA5E504FEACE2EB4F1FD0C88BFBCF5E06F1ED8BEF1004F9C
:2080000008BF5FEA500E50F1000041EB045170BD06F0004646EA010140EA020081EA0301FA
:20802000B4EB5C04C2BFD4EB0C0541EA045170BD41F480114FF0000E013C00F3AB8014F1D0
:20804000360FDEBF002001F0004170BDC4F10004203C35DA0C341BDC04F11404C4F120057D
:2080600000FA05F320FA04F001FA05F240EA020001F0004221F0004110EBD37021FA04F60A
:2080800042EB06015EEA430E08BF20EAD37070BDC4F10C04C4F1200500FA04F320FA05F033
:2080A00001FA04F240EA020001F0004110EBD37041F100015EEA430E08BF20EAD37070BD26
:2080C000C4F1200500FA05F24EEA020E20FA04F301FA05F243EA020321FA04F001F0004117
:2080E00021FA04F220EA020000EBD3705EEA430E08BF20EAD37070BD94F0000F0FD101F0F7
:208100000046400041EB010111F4801F08BF013CF7D041EA060195F0000F18BF704703F0F5
:208120000046520043EB030313F4801F08BF013DF7D043EA0603704794EA0C0F0CEA13551D
:2081400018BF95EA0C0F0CD050EA410618BF52EA4306D1D181EA030101F000414FF0000073
:2081600070BD50EA410606BF1046194652EA430619D094EA0C0F02D150EA013613D195EA29
:208180000C0F05D152EA03361CBF104619460AD181EA030101F0004141F0FE4141F4700157
:2081A0004FF0000070BD41F0FE4141F4780170BD70B54FF0FF0C4CF4E06C1CEA11541DBFC6
:2081C0001CEA135594EA0C0F95EA0C0F00F0A7F8A4EB050481EA030E52EA03354FEA01317C
:2081E00000F088804FEA03334FF0805545EA131343EA12634FEA022245EA111545EA1065B7
:208200004FEA00260EF000419D4208BF964244F1FD0404F5407402D25B084FEA3202B61AEB
:2082200065EB03055B084FEA32024FF480104FF4002CB6EB020E75EB030E22BFB61A754646
:2082400040EA0C005B084FEA3202B6EB020E75EB030E22BFB61A754640EA5C005B084FEA68
:208260003202B6EB020E75EB030E22BFB61A754640EA9C005B084FEA3202B6EB020E75EB95
:20828000030E22BFB61A754640EADC0055EA060E18D04FEA051545EA16754FEA06164FEA85
:2082A000C30343EA52734FEAC2025FEA1C1CC0D111F4801F0BD141EA00014FF000004FF0CD
:2082C000004CB6E711F4801F04BF01430020B4F1FD0C88BFBCF5E06F3FF6AFAEB5EB030CB4
:2082E00004BFB6EB020C5FEA500C50F1000041EB045170BD0EF0004E4EEA113114EB5C0453
:20830000C2BFD4EB0C0541EA045170BD41F480114FF0000E013C90E645EA060E8DE60CEAED
:20832000135594EA0C0F08BF95EA0C0F3FF43BAF94EA0C0F0AD150EA01347FF434AF95EA06
:208340000C0F7FF425AF104619462CE795EA0C0F06D152EA03353FF4FDAE1046194622E772
:2083600050EA410618BF52EA43067FF4C5AE50EA41047FF40DAF52EA43057FF4EBAE12E703
:208380004FF0FF3C06E000BF4FF0010C02E000BF4FF0010C4DF804CD4FEA410C7FEA6C5CB8
:2083A0004FEA430C18BF7FEA6C5C1BD001B050EA410C0CBF52EA430C91EA030F02BF90EAEC
:2083C000020F0020704710F1000F91EA030F58BF994208BF90422CBFD8176FEAE37040F0D7
:2083E000010070474FEA410C7FEA6C5C02D150EA013C07D14FEA430C7FEA6C5CD6D152EA50
:20840000033CD3D05DF8040B704700BF8446104662468C461946634600E000BF01B5FFF7B3
:20842000B7FF002848BF10F1000F01BD4DF808EDFFF7F4FF0CBF012000205DF808FB00BF43
:208440004DF808EDFFF7EAFF34BF012000205DF808FB00BF4DF808EDFFF7E0FF94BF012035
:2084600000205DF808FB00BF4DF808EDFFF7CEFF94BF012000205DF808FB00BF4DF808EDE3
:20848000FFF7C4FF34BF012000205DF808FB00BF4A0011D212F5001211D20DD56FF478737F
:2084A000B3EB62520ED44FEAC12343F0004343EA505323FA02F070474FF00000704750EA2F
:2084C000013002D14FF0FF3070474FF0000070474FEA4102B2F1E04324BFB3F5001CDCF1C7
:2084E000FE5C0DD901F0004C4FEAC0024CEA5070B2F1004F40EB830008BF20F001007047DF
:2085000011F0804F21D113F13872BCBF01F00040704741F480114FEA5252C2F11802C2F165
:20852000200C10FA0CF320FA02F018BF40F001004FEAC1234FEAD32303FA0CFC40EA0C006B
:2085400023FA02F34FEA4303CCE77FEA625307D150EA01331EBF4FF0FE4040F440007047EE
:2085600001F0004040F0FE4040F40000704700BF80F0004002E000BF81F0004142001FBF8F
:208580005FEA410392EA030F7FEA226C7FEA236C6AD04FEA1262D2EB1363C1BFD2184140CC
:2085A00048404140B8BF5B42192B88BF704710F0004F40F4000020F07F4018BF404211F0B0
:2085C000004F41F4000121F07F4118BF494292EA030F3FD0A2F1010241FA03FC10EB0C006F
:2085E000C3F1200301FA03F100F0004302D5494260EB4000B0F5000F13D3B0F1807F06D382
:2086000040084FEA310102F10102FE2A51D2B1F1004F40EBC25008BF20F0010040EA030033
:208620007047490040EB000010F4000FA2F10102EDD1B0FA80FCACF1080CB2EB0C0200FA2C
:208640000CF0AABF00EBC25052421843BCBFD0401843704792F0000F81F4000106BF80F4EC
:2086600000000132013BB5E74FEA41037FEA226C18BF7FEA236C21D092EA030F04D092F0D7
:20868000000F08BF0846704790EA010F1CBF0020704712F07F4F04D1400028BF40F0004087
:2086A000704712F100723CBF00F50000704700F0004343F0FE4040F4000070477FEA22626B
:2086C00016BF08467FEA23630146420206BF5FEA412390EA010F40F4800070474FF0000354
:2086E00004E000BF10F0004348BF40425FEA000C08BF704743F0964301464FF000001CE0AA
:2087000050EA010208BF70474FF000030AE000BF50EA010208BF704711F0004302D540425B
:2087200061EB41015FEA010C02BF84460146002043F0B64308BFA3F18053A3F50003BCFAB8
:208740008CF2083AA3EBC25310DB01FA02FC634400FA02FCC2F12002BCF1004F20FA02F254
:2087600043EB020008BF20F00100704702F1200201FA02FCC2F1200250EA4C0021FA02F2C2
:2087800043EB020008BF20EADC7070474FF0FF0C1CEAD0521EBF1CEAD15392EA0C0F93EA48
:2087A0000C0F6FD01A4480EA010C400218BF5FEA41211ED04FF0006343EA501043EA51111A
:2087C000A0FB01310CF00040B1F5000F3EBF490041EAD3715B0040EA010062F17F02FD2AA5
:2087E0001DD8B3F1004F40EBC25008BF20F00100704790F0000F0CF0004C08BF49024CEAA6
:20880000502040EA51207F3AC2BFD2F1FF0340EAC250704740F400004FF00003013A5DDC71
:2088200012F1190FDCBF00F000407047C2F10002410021FA02F1C2F1200200FA02FC5FEA71
:20884000310040F1000053EA4C0308BF20EADC70704792F0000F00F0004C02BF400010F484
:20886000000F013AF9D040EA0C0093F0000F01F0004C02BF490011F4000F013BF9D041EA92
:208880000C018FE70CEAD15392EA0C0F18BF93EA0C0F0AD030F0004C18BF31F0004CD8D102
:2088A00080EA010000F00040704790F0000F17BF90F0004F084691F0000F91F0004F14D0A0
:2088C00092EA0C0F01D142020FD193EA0C0F03D14B0218BF084608D180EA010000F00040B9
:2088E00040F0FE4040F40000704740F0FE4040F4400070474FF0FF0C1CEAD0521EBF1CEA31
:20890000D15392EA0C0F93EA0C0F69D0A2EB030280EA010C49024FEA402037D04FF08053C5
:2089200043EA111143EA10130CF000408B4238BF5B0042F17D024FF4000C8B4224BF5B1A17
:2089400040EA0C00B3EB510F24BFA3EB510340EA5C00B3EB910F24BFA3EB910340EA9C008F
:20896000B3EBD10F24BFA3EBD10340EADC001B0118BF5FEA1C1CE0D1FD2A3FF650AF8B42E1
:2089800040EBC25008BF20F0010070470CF0004C4CEA50207F32C2BFD2F1FF0340EAC250EA
:2089A000704740F400004FF00003013A37E792F0000F00F0004C02BF400010F4000F013A15
:2089C000F9D040EA0C0093F0000F01F0004C02BF490011F4000F013BF9D041EA0C0195E7F2
:2089E0000CEAD15392EA0C0F08D142027FF47DAF93EA0C0F7FF470AF084676E793EA0C0F9D
:208A000004D14B023FF44CAF08466EE730F0004C18BF31F0004CCAD130F000427FF45CAF38
:208A200031F000437FF43CAF5FE700BF4FF0FF3C06E000BF4FF0010C02E000BF4FF0010C17
:208A40004DF804CD4FEA40024FEA41037FEA226C18BF7FEA236C11D001B052EA530C18BF3E
:208A600090EA010F58BFB2EB030088BFC81738BF6FEAE17018BF40F0010070477FEA226C38
:208A800002D15FEA402C05D17FEA236CE4D15FEA412CE1D05DF8040B704700BF8446084672
:208AA0006146FFE70FB5FFF7C9FF002848BF10F1000F0FBD4DF808EDFFF7F4FF0CBF01208D
:208AC00000205DF808FB00BF4DF808EDFFF7EAFF34BF012000205DF808FB00BF4DF808EDC1
:208AE000FFF7E0FF94BF012000205DF808FB00BF4DF808EDFFF7D2FF94BF012000205DF80C
:208B000008FB00BF4DF808EDFFF7C8FF34BF012000205DF808FB00BF4FEA4002B2F1FE4FE6
:208B20000FD34FF09E03B3EB12620DD94FEA002343F0004310F0004F23FA02F018BF4042F2
:208B400070474FF00000704712F1610F01D1420205D110F0004008BF6FF0004070474FF06D
:208B600000007047014B1868704700BF3407002008B5074B044613B10021AFF30080054BF1
:208B80001868836A03B198472046FCF7EBF900BF000000003CA4000870B50E4B0E4D0024F4
:208BA000ED1AAD101E46AC4204D056F8242090470134F8E700F02AFC084D094B0024ED1A64
:208BC000AD101E46AC4204D056F8242090470134F8E770BD189400081894000834940008D0
:208BE00018940008024B0146186800F059B800BF3407002010B50023934203D0CC5CC454C2
:208C00000133F9E710BD02440346934202D003F8011BFAE77047000030B500293CD051F82B
:208C2000042C0B1F1D49002AB8BF9B180A680C4612B95A600B6030BD93420DD219685818DA
:208C4000904203D15A581144426819605A60236030BD994203D80A4651680029F9D11468EC
:208C600015199D420AD11B682344D0188842136012D10868034413604B680CE002D90C2347
:208C8000036030BD18681C188C4203D10C684968204418605960536030BD00BF40120020A3
:208CA00070B5CD1C25F0030508350C2D38BF0C25002D06463FDB8D423DD3214B1C6818462B
:208CC0002146A1B10B685B1B0ED40B2B03D90B60CC18CD501FE08C4202D1626802601AE0CC
:208CE0004B6863600C4616E00C464968E9E7154C23681BB9304600F027F820602946304639
:208D000000F022F8431C014615D0C41C24F0030484420AD1256004F10B00231D20F0070046
:208D2000C31A0BD05A42E25070BD3046611A00F00BF80130EED10C233360002070BD00BFDE
:208D4000401200203C12002038B5064C0023054608462360FCF7E4F8431C02D1236803B175
:208D60002B6038BD841200200EB400B54FF402719CB0ADF814106FF00041049107914FF669
:208D8000FF711DABADF81610084953F8042B02900690086802A9019300F06EF8029B002219
:208DA0001A701CB05DF804EB03B0704734070020034613F8012B002AFBD1181A01387047BC
:208DC0002DE9F0478D688146AB420C4692461F4643D38B8913F4906F3DD0266809690222AD
:208DE000C1EB0608666906EB460696FBF2F608F101023A44964238BF16465B050FD53146D4
:208E0000FFF74EFF054698B121694246FFF7F2FEA38923F4906343F08003A38113E0324608
:208E200000F0C5FA054670B948462169FFF7F4FE0C23C9F80030A3894FF0FF3043F04003DF
:208E4000A381BDE8F087256166614544C8EB06062560A6603D46AF4200D23D462A462068F1
:208E6000514600F089FAA36800205B1BA36023681D442560BDE8F0872DE9F0439DB003938B
:208E80008B8907461C060D4616460CD50B6953B94021FFF705FF2860286110B90C233B6040
:208EA000C7E040236B610023099320238DF8293030238DF82A3033461C4613F8012B1AB9E5
:208EC000B4EB06090FD002E0252AF5D1F8E73846294632464B46FFF773FF013000F0A4808C
:208EE000099B4B4409932378002B00F09D8000234FF0FF3204930793059206938DF85330D4
:208F00001A9304F101094D4E4C4630462178052200F024FA09F10109049B28B1861B0120F6
:208F2000B04003430493EEE7D90644BF20228DF853201A0744BF2B228DF8532022782A2A1C
:208F400002D0079B21460EE0039A111D12680391002A01DB079204E0524243F00203079287
:208F6000049301340AE00C4622780131303A092A03D80A2000FB0323F5E7079323782E2BF0
:208F800019D163782A2B09D1039B02341A1D1B680392002BB8BF4FF0FF330BE0611C00231C
:208FA0000C4622780131303A092A03D80A2000FB0323F5E70593224E21783046032200F0C8
:208FC000CDF930B1861B4020B040049B01340343049321781B480622661C8DF8281000F0F5
:208FE000BDF988B1184B33B9039B073323F007030833039314E003AB0093384604A92A469D
:20900000124BAFF3008007E003AB0093384604A92A460E4B00F08EF8B0F1FF3F804603D0C7
:20902000099B4344099346E7AB895B0601D4099801E04FF0FF301DB0BDE8F08340A4000811
:2090400046A400084AA4000800000000C18D00082DE9F84315461F468A680B6906469A4233
:20906000A8BF13462B6091F843200C46DDF820800AB101332B602368990602D52B680233AF
:209080002B60236813F006091DD094F843302268003318BF012392061FD5E118302081F8B6
:2090A00043005A1C94F845102244023382F8431013E03046394604F119020123C04701305A
:2090C00007D009F10109E2682B68D31A9945F0DBDBE74FF0FF30BDE8F8833046394604F108
:2090E0004302C0470130F4D023682A6803F00603E168042B08BFC2EB01052369A2680CBFC3
:2091000025EAE57500259A42C4BFC3EB0203ED184FF00009A9450ADA3046394604F11A028A
:209120000123C0470130D4D009F10109F2E70020BDE8F8832DE9FF470E7E80466E2E0C4676
:2091400091469A460C9D01F1430000F0A58011D8632E22D009D8002E00F0AF80582E40F015
:20916000BF8081F845607B4A4FE0642E1ED0692E1CD0B5E0732E00F0A48009D86F2E2BD0D8
:20918000702E40F0AD800B6843F020030B6038E0752E21D0782E34D0A2E02B6801F14207FA
:2091A0001A1D1B682A6081F842309DE022682B6812F0800F03D01A1D2A601D6805E0510600
:2091C000F9D51A1D2A60B3F90050002D39DA2D236D4284F8433034E022682B6812F0800F14
:2091E00003D01A1D2A601D6804E05206F9D51A1D2A601D88237E574A6F2B14BF0A230823DF
:209200001BE07823544A84F845302368296813F0800F01F104062E6001D00D6802E05F0664
:20922000FBD50D88DE0744BF43F0200323601DB9236823F0200323601023002184F84310CB
:2092400001E0444A0A236668002EA66003DB216821F00401216005B96EB104F14201B5FBAD
:20926000F3F603FB1655555D0F4601F801593546002EF4D100E00746082B0AD12368DD072A
:2092800007D5626823699A4203DC302307F8013C013FC01B20612CE009682B6811F0800F16
:2092A000626904D0191D29601B681A6005E04906F8D5191D29601B681A8000232361074682
:2092C00017E02B681A1D2A601F683846FFF770FD63682061984288BF23612369636005E0B6
:2092E00004F1420784F8426001232361002384F84330CDF800A04046214603AA4B46FFF7D2
:20930000A7FE013002D14FF0FF301FE0404649463A462369D0470130F5D023689B0705D403
:20932000E068039B9842B8BF18460FE00025E268039BD31A9D42F3DA4046494604F11902DE
:209340000123D0470130DED00135F0E704B0BDE8F08700BF51A4000862A4000810B5C9B20C
:2093600002449042034605D01C7801308C42F8D1184610BD002010BD814270B501D3002364
:209380000EE08C18A042FAD28518134613F1FF3305D351426618F65C2944CE54F6E770BD8D
:2093A000934203D0CC5CC4540133F9E770BDF8B5064614460D4621B91146BDE8F840FFF7DA
:2093C0006FBC1AB9FFF728FC2046F8BD00F015F8A0420ED230462146FFF762FC074650B11C
:2093E00029462246FFF706FC30462946FFF714FC01E02846F8BD3846F8BD51F8040C0028FB
:2094000002DA04390B58184404387047F8B500BFF8BC08BC9E467047B96F00081121000898
:20942000D13400080D4A00086D4F0008056F000891710008F8B500BFF8BC08BC9E467047F7
:20944000ED2000080000000064BAFF7F01000000000000000000000020212223242526273E
:209460000001020304050607101112131415161718191A1B1C1D1E1F2C00C2010000000861
:2094800002030000420000001D35000800000000AD35000800000000000000000000000041
:2094A00055360008113600085C000020DD35000800000000400000080000000000000000EC
:2094C0001000000BA9360008000000004000000040000000400000000003000000000000C7
:2094E00000000000000000000000000000000000000000000000000000000000000000006C
:2095000000000000000000000000000000000000000000000000000000000000000000004B
:2095200000000000000000000000000000000000000000000000000000000000000000002B
:2095400000000000000000000000000000000000000000000000000000000000000000000B
:2095600000000000000000000000000000000000500B00200000000032010020120000000B
:2095800000011201000200000140AF1E2400000201020001F4010000B49E0008040000002A
:2095A000789E000800000000429E00080000000000000000000000000300000088000020FA
:2095C0000000000000000002000400060101000019000000694500080000000069440008F9
:2095E000000000000000000039460008BD440008C5450008A801002089440008000000002B
:209600004000000B40000000C19E000809000000E49E0008050C0901A1018503150026FF46
:209620000319002AFF03751095018100C0000000D49E0008DC9E0008EC9E000805010902E7
:20964000A10185010901A10005091901290815002501950875018102050109300931093853
:209660001581257F750895038106C0C005010904A1018514150025017501952005091901B8
:2096800029208102150025073500463B0175049501651405010939814205010901A10015AD
:2096A0000026FF03750A950409300931093309348102C0150026FF03750A9502093609366A
:2096C0008102C005010906A1018502050719E029E71500250175019508810295017508818F
:2096E0000395067508150025650507190029658100050819012908950875019102C00000BE
:20970000000010000500008000000100B00200200028014001000000002401400012000000
:2097200000000000000000000000000000000000C0020020C8020020000002400700000014
:20974000000000000B000000000000000C000000000000000D000000000000000E000000D7
:20976000000000000F00000000000000100000000000000011000000E80200200008014066
:209780000B000000000C01400C010000001001400D020000001401400E030000005400400A
:2097A00000000000000000000000000034030020000000000000000000000706121F2000F4
:2097C0000000000000000000000000000000000000000000005800400000000000000000F1
:2097E0000000000034030020000000000000000000000B0A132122000000000000000000A7
:209800000000000000000000000000001C1002401810024014100240101002400C1002404A
:209820001C1002401810024014100240000400401C01000000000000000000000000000089
:2098400000000000000000000000000000000000000800401D0100000000000000000000A2
:209860000000000000000000000000000000000000000000002C01401A0000000000000061
:20988000000000000000000000000000000000000000000000000000000000000000004088
:2098A0001B010000000000000000000000000000000000000000000000000000000000008C
:2098C0007C04002010050020A405002000380140B40F0020A80F002020AA440000000000A9
:2098E000000000000000000000000000000000000000000000000000000000000000000068
:20990000000000000000000000000000000000000000000000000000000000000000000047
:20992000000000000000000000000000000000000000000000000000000000000000000027
:209940000000000000000000000000000000000000000000000000000000000028250000BA
:2099600000440040C00F0020D80F00201055220000000000000000000000000000000000E6
:209980000000000000000000000000000000000000000000000000000000000000000000C7
:2099A0000000000000000000000000000000000000000000000000000000000000000000A7
:2099C000000000000000000000000000000000000000000000000000000000000000000087
:2099E000000000000000000000000000000000002926000000480040CC0F0020E40F002082
:209A00001055220000000000000000000000000000000000000000000000000000000000BF
:209A2000000000000000000000000000000000000000000000000000000000000000000026
:209A4000000000000000000000000000000000000000000000000000000000000000000006
:209A60000000000000000000000000000000000000000000000000000000000000000000E6
:209A8000000000002A2700003C06002000BF0000000000000000000000002D0078A3000804
:209AA00043000000496000082D610008BD6B0008BD6B0008315F0008855F0008D55F0008FC
:209AC0003D60000831600008116000080000000040000000BBA300080400000054A3000826
:209AE0001200000048A300080C00000000C2010000000800BD6B0008E55F0008BD6B0008DE
:209B0000BD6B0008BD6B0008BD6B0008BD6B0008BD6B00080160000866A3000812000000C9
:209B200004010100000000000000000000000000000000000000000000000000000000001F
:209B40000000000038A4000800000000000000000000000000000000000000000000000021
:209B60000000000000000000000000000000000000000000000000000000000000000000E5
:209B800000000000D40600200000F401D0072564202564204D256420707265737365640AB7
:209BA000002564202564204D25642072656C65617365640A0042256420707265737365642D
:209BC0000A00436C6F636B776F726B50490075436F6E736F6C650032303233303731330059
:209BE000DA00D900D800D700EE00EF00F000F10081008500800084008200F5008600F70047
:209C0000FD00D300D600D200D500EE00EF00F000F10000010001800084008700F500860031
:209C2000F700FD00050C0901A1018503150026FF0319002AFF03751095018100C0050109FE
:209C400006A1018502050719E029E71500250175019508810295017508810395067508152B
:209C60000025650507190029658100050819012908950875019102C005010904A10185141A
:209C800015002501750195200509190129208102150025073500463B0175049501651405E5
:209CA000010939814205010901A100150026FF03750A950409300931093309348102C01554
:209CC0000026FF03750A9502093609368102C005010902A10185010901A100050919012950
:209CE000081500250195087501810205010930093109381581257F750895038106C0C0007B
:209D0000E800E900FA0060005B005D002D003D003100320033003400350036003700380052
:209D200039003000B100B300FFFFFFFFFFFFFFFF71007700650072007400790075006900D4
:209D40006F0070006100730064006600670068006A006B006C007A00780063007600620049
:209D60006E006D002C002E002F005C003B002700B200B000F400F4002000FFFFFFFFFFFF5D
:209D8000CE00D000FB0060005B005D00CC00CD00C200C300C400C500C600C700C800C9004D
:209DA000CA00CB00FE00C100FFFFFFFFFFFFFFFF710077006500720074007900D300D10007
:209DC0006F00700061007300640066006700D200D500D6006C007A00780063007600620089
:209DE0006E006D00F900F8002F005C003B002700D400B000F400F400FF00FFFFFFFFFFFF45
:209E0000080B00020202010209040000010202010005240001100524010301042402060576
:209E200024060001070580031000FF09040100020A00000007050002400000070580024023
:209E400000004D61706C650009020000000100C032000000BD6B0008713A0008BD6B000802
:209E6000BD6B0008BD6B0008B13A0008BD6B0008BD6B0008D93A00084C6561664C6162731A
:209E800000000000813B0008093C0008BD6B0008BD6B00089D390008093A0008E93A0008FD
:209EA000753B0008693B0008053B0008000000004000000004030904090400000103010090
:209EC000000921100100012200000705800340000A0000001C020020570000007302002021
:209EE0003B000000C401002019000000EC0100203000000000000000000000002A2B28006F
:209F000000000000000000000000000000000000000000002C9EB4A0A1A2A434A6A7A5AE68
:209F2000362D3738271E1F20212223242526B333B62EB7B89F8485868788898A8B8C8D8E3B
:209F40008F909192939495969798999A9B9C9D2F3130A3AD350405060708090A0B0C0D0EBF
:209F60000F101112131415161718191A1B1C1DAFB1B0B500000000000000000000000000D2
:209F8000854700085D6F00083D6F00080948000867480008654700080000000000000000A1
:209FA000254C00083D4C00083D6F0008454A0008674A0008494A0008C54B000800000000E0
:209FC0002C0300204C040020C8020020000100002C0300204C040020C8020020010201002A
:209FE0002C0300204C040020C8020020020302002C0300204C040020C802002003040300FE
:20A000002C03002000000000C8020020040004002C03002000000000C802002005000500BC
:20A020002C030020DC030020C8020020060106002C030020DC030020C80200200702070093
:20A040002C03002024040020000000000801FF002C03002024040020000000000902FF00C0
:20A060002C03002024040020000000000A03FF002C03002024040020000000000B04FF0098
:20A080002C03002000000000000000000C00FF002C03002000000000000000000D00FF000B
:20A0A0002C03002000000000000000000E00FF002C03002000000000000000000F00FF00E7
:20A0C00034030020DC030020C80200200003080034030020DC030020C802002001040900E7
:20A0E0003403002000000000000000000200FF003403002000000000000000000300FF00AF
:20A100003403002000000000000000000400FF003403002000000000000000000500FF008A
:20A120003403002000040020000000000601FF003403002000040020000000000702FF001B
:20A140003403002000040020000000000803FF003403002000040020000000000904FF00F3
:20A160003403002000000000000000000A00FF003403002000000000000000000B00FF001E
:20A180003403002000000000000000000C00FF003403002000000000000000000D00FF00FA
:20A1A0003403002000000000000000000E00FF003403002000000000000000000F00FF00D6
:20A1C0003C03002000000000C802002000000A003C03002000000000C802002001000B00D7
:20A1E0003C03002000000000C802002002000C003C03002000000000C802002003000D00AF
:20A200003C03002000000000C802002004000E003C03002000000000C802002005000F0086
:20A220003C03002000000000000000000600FF003C03002000000000000000000700FF0055
:20A240003C03002000000000000000000800FF003C03002000000000000000000900FF0031
:20A260003C03002000000000000000000A00FF003C03002000000000000000000B00FF000D
:20A280003C03002000000000000000000C00FF003C03002000000000000000000D00FF00E9
:20A2A0003C03002000000000000000000E00FF003C03002000000000000000000F00FF00C5
:20A2C0004403002000000000000000000200FF002C030020340300200109010A010F01004A
:20A2E000001B020600000200000002040000010201030104010500000000000000150016F6
:20A30000001C0000010C000E00000202010B000000010002000000000000000000000000F3
:20A320000000000000000000010E00110012000000000017F00000000007000000380000A5
:20A340000000C00000C000000C034D00610070006C00650012034C006500610066004C00A6
:20A360006100620073001201000202000040AF1E040000020102000109024300020100C068
:20A38000320904000001020201000524000110052401030104240206052406000107058222
:20A3A000034000FF09040100020A000000070503024000000705810240000004030904000D
:20A3C0000000000000000000256E00085D6F00083D6F0008DD6D0008A36D0008E96D000892
:20A3E0000B6E00080000000000000000000000007B6F00085D6F00083D6F00080000000062
:20A400000000000000000000297100083F7100083D6F000889700008AB7000088D70000805
:20A4200075710008000000007371727400000000737172746600000043000000D4060020F7
:20A44000232D302B2000686C4C0065666745464700303132333435363738394142434445B1
:20A46000460030313233343536373839616263646566000050940008FFFFFFFFFFFFFFFF50
:20A48000FFFFFFFFFFFFFFFFFFFFFFFFFFFFFFFFFFFFFFFFFFFFFFFFFFFFFFFFFFFFFFFFDC
:20A4A000FFFFFFFFFFFFFFFFFFFFFFFFFFFFFFFFFFFFFFFFFFFFFFFFFFFFFFFFFFFFFFFFBC
:20A4C000FFFFFFFFFFFFFFFFFFFFFFFFFFFFFFFFFFFFFFFFFFFFFFFFFFFFFFFFFFFFFFFF9C
:20A4E000FFFFFFFFFFFFFFFFFFFFFFFFFFFFFFFFFFFFFFFFFFFFFFFFFFFFFFFFFFFFFFFF7C
:20A50000FFFFFFFFFFFFFFFFFFFFFFFFFFFFFFFFFFFFFFFFFFFFFFFFFFFFFFFFFFFFFFFF5B
:20A52000FFFFFFFFFFFFFFFFFFFFFFFFFFFFFFFFFFFFFFFFFFFFFFFFFFFFFFFFFFFFFFFF3B
:20A54000FFFFFFFFFFFFFFFFFFFFFFFFFFFFFFFFFFFFFFFFFFFFFFFFFFFFFFFFFFFFFFFF1B
:20A56000FFFFFFFFFFFFFFFFFFFFFFFFFFFFFFFFFFFFFFFFFFFFFFFFFFFFFFFFFFFFFFFFFB
:20A58000FFFFFFFFFFFFFFFFFFFFFFFFFFFFFFFFFFFFFFFFFFFFFFFFFFFFFFFFFFFFFFFFDB
:20A5A000FFFFFFFFFFFFFFFFFFFFFFFFFFFFFFFFFFFFFFFFFFFFFFFFFFFFFFFFFFFFFFFFBB
:20A5C000FFFFFFFFFFFFFFFFFFFFFFFFFFFFFFFFFFFFFFFFFFFFFFFFFFFFFFFFFFFFFFFF9B
:20A5E000FFFFFFFFFFFFFFFFFFFFFFFFFFFFFFFFFFFFFFFFFFFFFFFFFFFFFFFFFFFFFFFF7B
:20A60000FFFFFFFFFFFFFFFFFFFFFFFFFFFFFFFFFFFFFFFFFFFFFFFFFFFFFFFFFFFFFFFF5A
:20A62000FFFFFFFFFFFFFFFFFFFFFFFFFFFFFFFFFFFFFFFFFFFFFFFFFFFFFFFFFFFFFFFF3A
:20A64000FFFFFFFFFFFFFFFFFFFFFFFFFFFFFFFFFFFFFFFFFFFFFFFFFFFFFFFFFFFFFFFF1A
:20A66000FFFFFFFFFFFFFFFFFFFFFFFFFFFFFFFFFFFFFFFFFFFFFFFFFFFFFFFFFFFFFFFFFA
:20A68000FFFFFFFFFFFFFFFFFFFFFFFFFFFFFFFFFFFFFFFFFFFFFFFFFFFFFFFFFFFFFFFFDA
:20A6A000FFFFFFFFFFFFFFFFFFFFFFFFFFFFFFFFFFFFFFFFFFFFFFFFFFFFFFFFFFFFFFFFBA
:20A6C000FFFFFFFFFFFFFFFFFFFFFFFFFFFFFFFFFFFFFFFFFFFFFFFFFFFFFFFFFFFFFFFF9A
:20A6E000FFFFFFFFFFFFFFFFFFFFFFFFFFFFFFFFFFFFFFFFFFFFFFFFFFFFFFFFFFFFFFFF7A
:20A70000FFFFFFFFFFFFFFFFFFFFFFFFFFFFFFFFFFFFFFFFFFFFFFFFFFFFFFFFFFFFFFFF59
:20A72000FFFFFFFFFFFFFFFFFFFFFFFFFFFFFFFFFFFFFFFFFFFFFFFFFFFFFFFFFFFFFFFF39
:20A74000FFFFFFFFFFFFFFFFFFFFFFFFFFFFFFFFFFFFFFFFFFFFFFFFFFFFFFFFFFFFFFFF19
:20A76000FFFFFFFFFFFFFFFFFFFFFFFFFFFFFFFFFFFFFFFFFFFFFFFFFFFFFFFFFFFFFFFFF9
:20A78000FFFFFFFFFFFFFFFFFFFFFFFFFFFFFFFFFFFFFFFFFFFFFFFFFFFFFFFFFFFFFFFFD9
:20A7A000FFFFFFFFFFFFFFFFFFFFFFFFFFFFFFFFFFFFFFFFFFFFFFFFFFFFFFFFFFFFFFFFB9
:20A7C000FFFFFFFFFFFFFFFFFFFFFFFFFFFFFFFFFFFFFFFFFFFFFFFFFFFFFFFFFFFFFFFF99
:20A7E000FFFFFFFFFFFFFFFFFFFFFFFFFFFFFFFFFFFFFFFFFFFFFFFFFFFFFFFFFFFFFFFF79
:20A800000B9D02350B95DDF824C01CF0840CCDF84CC040F090820F9DDDF82CC0CCEB050B1D
:20A82000BBF1000F40F38782BBF1100F2D992C9ADFF8A0A12CDD1B97304657461025CA469F
:20A840000C9EA1460D9C06E0ABF1100BBBF1100F00F1080017DD01321031072A2D912C9248
:20A8600007604560F0DD204631462BAA02F05EFD00287FF43BAFABF1100BBBF1100F2D9933
:20A880002C9A38A8E7DC4C46D146BA461B9F064601320BEB010C072ACDF8B4C02C9286E8D4
:20A8A000000C00F31A849DF88FA00836BAF1000F0FD02C9B0CF1010C01330DF18F010122AA
:20A8C000072BCDF8B4C02C9386E8060000F3A4830836129B73B12C9B0CF1020C013324A9DE
:20A8E0000222072BCDF8B4C02C9386E8060000F387830836139D802D00F0CA820A9DC4EB6C
:20A90000050ABAF1000F3BDDBAF1100F2C9B304D2BDD0A9432464FF0100B2E4661460D9C0C
:20A920000C9D06E0AAF1100ABAF1100F02F1080217DD01331031072B2D912C9382E8400842
:20A94000F0DD204629462BAA02F0F0FC00287FF4CDAEAAF1100ABAF1100F2D992C9B38AA9E
:20A96000E7DC0A9C35468C4616460133D444072BCDF8B4C02C9386E8200400F335830836D4
:20A98000099DED0500F124822C9BA4440133072BCDF8B4C0376074602C9300F30F8308364D
:20A9A000099C630749D50F9D0B982C1A002C44DD102C2C9BDFF81CA02BDD57461025624670
:20A9C000DDF83080DDF834A00BE000BF84F2000850F20008A4F20008103C102C06F10806AC
:20A9E00015DD01331032072B2D922C9337607560F2DD504641462BAA02F098FC00287FF4F1
:20AA000075AE103C102C2D9A2C9B38AEE9DC9446BA460133A444072BCDF8B4C02C93C6F874
:20AA200000A0746009DD0D980C992BAA02F07EFC00287FF45BAEDDF8B4C00E9C0B980F9D4B
:20AA4000A842ACBF241864190E94BCF1000F40F0C18200232C9338AE56E599F80080002AD9
:20AA60007FF488AD202285E5099D45F00105099599F800807EE5099D45F08005099599F800
:20AA8000008077E50024A8F130030F94214619F8018B01EB810103EB4101A8F13003092BA5
:20AAA000F5D90F9168E5DDF824C08DF88F204CF0100CCDF824C0099CA50640F1B280109D8D
:20AAC000E91D21F00701D1E900230831109114461D46002A73F1000CC0F294839DF88FA0BC
:20AAE000012359E6099DB64CAF068DF88F201A943FF52FAE099DED0640F14384DDF840C03D
:20AB00000025DCF800400CF1040CCDF840C02BE6DDF824C08DF88F201CF0200F00F040843D
:20AB2000109C21680E9CE5172B46109D224604351095C1E90023E7E4109C4FF0000A2768BA
:20AB40008DF88FA0251D002F00F0E9850A9C3846002CC0F29B855146224602F093F80028AC
:20AB600000F013860A9CC01BA042B8BF0446109524EAE475CDF828A0CDF850A00B959DF8A5
:20AB80008FA032E6DDF824C04CF0400CCDF824C099F80080EEE499F800804B46B8F16C0FDB
:20ABA00000F07F84099D45F010050995E2E4109C109D24682B1D002C0F94FFF67DAD109390
:20ABC00099F80080D6E4109BDDF824C0109D7D4804351C684FF0780830234CF0020C109516
:20ABE0008DF89030CDF824C000258DF891801A900223CDE5109B109D1A68012400230435D0
:20AC00009A460B948DF8B82010958DF88F300A9314932EAFEFE5099C8DF88F20A5063FF5C2
:20AC20004EAFDDF824C01CF0100F40F0DF82DDF824C01CF0400F00F0D982DDF840C0BCF9B9
:20AC400000400CF1040CE51722462B46CDF840C03FE799F800802B228CE4099D45F0080531
:20AC6000099599F8008085E4109D8DF88F20EB1D23F0070303F1080CCDF840C0D3E90045E8
:20AC8000CDE91645DDE91601FDF7DCFB0128DDE9160140F05C8300220023FEF75FF900282C
:20ACA00040F063859DF88FA003250B95099D464F25F08005454B0024099500250A94B8F15D
:20ACC000470FD8BF1F46032414958EE5DDF824C04CF0200CCDF824C099F800804AE4109C2A
:20ACE000E31D23F0070303F108051095D3E9004500234DE5109DEB1D23F0070303F1080C61
:20AD0000D3E90045CDF840C0012341E58DF88F20B8F1000F3FF4E3AC00234FF0010C9A4626
:20AD2000CDF82CC08DF8B8808DF88F300A93149364462EAF5FE5DDF8B4C0B7E5012B00F051
:20AD4000EC80022B0DF1DF0318D1DDF868C0194604F00F0022091CF8000042EA05722B091C
:20AD6000087052EA03000F4614461D4601F1FF31EED1089DCDE91E23EC1B2DE5E00840EA62
:20AD8000457004F00702E908303250EA010C1F461A7004460D4603F1FF33EFD1099CCDE99A
:20ADA0001C01E007394640F1C180302A00F0BE80089D1F463023EC1B01F8013C0CE500BFCC
:20ADC00070F2000884F2000864F2000860F20008B8F1650F40F3AD80DDE916010022002334
:20ADE000CDF81CC0FEF7B0F8DDF81CC0002800F026812C9BAA4901330CF1010C0122072B58
:20AE0000CDF8B4C02C9386E8060000F3ED820836259B119CA34203DB099DEC077FF5C0AD7C
:20AE20002C9B189C0133159DA444072BCDF8B4C0356074602C9300F33E830836119D6C1E0C
:20AE4000002C7FF7ADAD102C2C9B964D40F3978110276246DDF83480DDF830A004E0083696
:20AE6000103C102C40F38A8101331032072B2D922C9386E8A000F2DD404651462BAA02F025
:20AE800055FA00287FF432AC2D9A2C9B38AEE7E70F9D0B98C0EB050ABAF1000F7FF72EAD94
:20AEA000BAF1100F2C9B7F4D2BDD129432464FF0100B2E4661460D9C0C9D06E0AAF1100AAD
:20AEC000BAF1100F02F1080217DD01331031072B2D912C9382E84008F0DD204629462BAA6A
:20AEE00002F024FA00287FF401ACAAF1100ABAF1100F2D992C9B38AAE7DC129C35468C464E
:20AF000016460133D444072BCDF8B4C02C9386E8200400F30F820836F0E4002D08BF0A2C0D
:20AF200080F03881303448AF07F8414D089DEC1B52E4119C012C2C9C40F3D28101340CF1C4
:20AF400001030122072C2D9337602C94726000F3D8810836159DDDF8608001343560189D3E
:20AF60009844072CCDF8B4802C94756000F3D5810836DDE9160100220023FDF7E5FF119D05
:20AF8000002840F0B9806B1E013401379844072C2C94CDF8B4803760736000F3E280083665
:20AFA000DDF864C00134199DC44427AB072CCDF8B4C02C9486E828007FF7F1AC0D980C99B4
:20AFC0002BAA02F0B3F900287FF490ABDDF8B4C038AEE5E40D980C992BAA02F0A7F9002857
:20AFE0003FF437ADFFF782BB0D980C992BAA02F09DF900287FF47AABDDF8B4C038AEBFE4CE
:20B000000D980C992BAA02F091F900287FF46EABDDF8B4C038AE6DE40D980C992BAA02F050
:20B0200085F900287FF462ABDDF8B4C038AE50E40A9C38AFFFF7D0BB0223FFF7A9BB259B3A
:20B04000002B40F3DD81119C149DDDF844A0AC42A8BF2C46002CBA440BDD2C9BA444013361
:20B06000072BCDF8B4C0376074602C9300F31E830836149D24EAE4742C1B002C40F3D78055
:20B08000102C2C9B074D40F3A3810A974FF010082F4662462546DDF834B00C9C09E000BF79
:20B0A000A0F2000850F200080836103D102D40F38B8101331032072B2D922C9386E8800190
:20B0C000F2DD584621462BAA02F030F900287FF40DAB2D9A2C9B38AEE7E70D980C992BAAF8
:20B0E00002F024F900287FF401AB9DF88FA0DDF8B4C038AEFFF7DABB6F1E002F7FF750AF4B
:20B10000102FAE4D23DD43464FF0100ADDF83480DDF830B004E0103F102F06F1080615DD6C
:20B1200001341033072C2D932C9486E82004F2DD404659462BAA02F0F9F800287FF4D6AA8B
:20B14000103F102F2D9B2C9C38AEE9DC98460134B844072CCDF8B4802C9486E8A0007FF7A7
:20B160001EAF0D980C992BAA02F0E0F800287FF4BDAADDF8B4802C9C38AE11E7944601335A
:20B18000A444072BCDF8B4C02C93356074607FF706AC13E70DF1DF0B204629460A22002306
:20B1A000FEF796FA30328BF80020204629460A220023FEF78DFA04460D4654EA050C5F46D4
:20B1C0000BF1FF3BE8D1089DEC1BFFF705BB109D01232C68043510950025FFF7D9BA109D80
:20B1E0002C68043510950025FFF7D2BA109D2C6804351095E51722462B46002A73F1000CA8
:20B20000BFF66CAC4FF02D0A644265EB45058DF88FA00123FFF7C0BA0D980C992BAA02F052
:20B2200085F800287FF462AADDF8B4C038AE149D259C2F44119DAC4242DB099DE9073FD474
:20B240001198C7EB0A05041BAC42B8BF2546002D0BDD2C9BAC440133072BCDF8B4C0376093
:20B2600075602C9300F34C82083625EAE575641B002C7FF795AB102C2C9B504D7FF77FAF2D
:20B2800010276246DDF83480DDF830A004E00836103C102C7FF772AF01331032072B2D92F9
:20B2A0002C9386E8A000F2DD404651462BAA02F03DF800287FF41AAA2D9A2C9B38AEE7E738
:20B2C000189D2C9BAC44159D01333560189D072BCDF8B4C075602C9300F3F4810836AFE797
:20B2E000099DEA073FF52AAE01340CF101080123072CCDF8B4802C94376073607FF74FAE83
:20B300002FE70D980C992BAA02F010F800287FF4EDA92D9B2C9C38AE1CE60D980C992BAA36
:20B3200002F004F800287FF4E1A9DDF8B4802C9C38AE1EE60D980C992BAA01F0F7FF002811
:20B340007FF4D4A9DDF8B4C038AEFFF7D7BAFDF779F8002840F0BB80099C194F194B4FF09F
:20B36000030C24F0800409940A90CDF82CC01490B8F1470FD8BF1F4664469DF88FA0FFF73B
:20B3800034BA099C640640F15081DDF840C00025BCF800400CF1040CCDF840C0FFF7E4B95B
:20B3A000DDF824C01CF0100F00F04681109C0E9D2368043410941D60FFF7A6B850F2000819
:20B3C0006CF2000868F200082C463D460A9F94460133A444072BCDF8B4C02C93356074607E
:20B3E0003FF71AAF083622E70D980C992BAA01F09DFF00287FF47AA9DDF8B4C038AE07E582
:20B400002C9AB74901320CF1010C0120072ACDF8B4C02C923160706000F3F78008361C4675
:20B420002CB9119D1DB9099DE8077FF5B9AA2C9B159D189901333560189D6144072B2D91FA
:20B4400075602C9300F3DE8106F108026442002C40F30B81102CA34D40F34881A34610262D
:20B460000C46DDF83480DDF830A006E00832ABF1100BBBF1100F40F3378101331034072B15
:20B480002D942C9382E86000F0DD404651462BAA01F04CFF00287FF429A92D9C2C9B38AA88
:20B4A000E5E7099C09F1010944F02004099493F80180FFF75FB80D980C992BAA01F036FFC4
:20B4C00000287FF413A9DDF8B4C038AEB6E40A9D28F0200A013500F0A580BAF1470F04D142
:20B4E0000A9D002D08BF01250A95DDF824C0DDE916234CF4807C002BCDF848C0C0F29C8131
:20B50000DDE91645CDE920454FF0000BB8F1660F00F09B81B8F1460F00F0A981BAF1450F64
:20B520000ABF0A9C0A9D651C022025A926AA29AB8DE821000392049302910D98DDE92023DD
:20B5400000F04EFBB8F1670F074602D0B8F1470F05D1DDF824C01CF0010F00F09C81BAF112
:20B56000460F07EB050400F01C81DDE9200100220023FDF7E9FC002840F00581299B9C4269
:20B5800006D930215A1C29921970299B9C42F9D8DB1BBAF1470F119300F0ED80B8F1650F39
:20B5A00040F3F281B8F1660F00F06881259C1494119C149DAC4200F33281DDF824C01CF0CE
:20B5C000010F40F0AD8125EAE5732C464FF06708BBF1000F40F0B280129D0B930995CDF8A9
:20B5E00028B09DF88FA0FFF700B90D984021FEF79DFB20602061002800F0BF81DDF830C04F
:20B600004023CCF81430FEF76FBF0D980C992BAA01F08CFE00287FF469A8259CDDF8B4C04C
:20B6200038AEFDE606240A945FE7109D2C68043510950025FFF798B8DDF824C01CF0400F95
:20B6400000F08780109C0E9D2368043410941D80FEF75ABF0D980C992BAA01F067FE0028ED
:20B660007FF444A82D992C9B38AADDF844C00133119C8C44072BCDF8B4C02C93176054601D
:20B680003FF79CAC02F10806FFF78AB9CDF828A0FEF7E4FE10950A9D20EAE07C0446CDF8CD
:20B6A0002CC014959DF88FA0FFF79FB80D980C992BAA01F03BFE00287FF418A8DDF8B4C0F7
:20B6C00038AED6E40D980C992BAA01F02FFE00287FF40CA8259CDDF8B4C038AEB0E500BFFA
:20B6E000A0F2000850F2000821465C4601332144072B2D912C9315605460ABDC0832B4E790
:20B700000D980C992BAA01F011FE00287EF4EEAF259C1199DDF8B4C00C1B38AEA5E50A9CE2
:20B72000BA46062C28BF062424EAE47C0A9714971095CDF82CC0974FFFF757B8129D4FF0DD
:20B740002D0A099500250B938DF88FA00A95FFF74FB8DDF840C00E9CDCF800300CF1040C71
:20B76000CDF840C01C60FEF7CFBE4FF02D0A8DF88FA0FFF799BA259BDC1C19DB0A9C9C4263
:20B7800016DB149314E7234602E724EAE47CCDF82CC00A9C10950A9014909DF88FA0FFF762
:20B7A00024B83B78302B00F0AD80259D2C44DCE6A8F10208591E00292591BABF49422D2341
:20B7C0002B2309298DF89C808DF89D3065DC302330318DF89E308DF89F1028AB119D27AA28
:20B7E000119C9A1A012D1992144440F3B7800134002524EAE4731495EAE6002481460A948C
:20B80000FEF7BABE0D980C992BAA01F08FFD00287EF46CAF259C2D992C9B38AA16E6149C8E
:20B82000119D002CD4BFC4F1020401242C4424EAE4734FF06708CBE61799169801F10041F6
:20B84000209021914FF02D0B60E60A9D032025A926AA29AB019500900392049302910D9803
:20B86000DDE9202300F0BCF90A9D074677E60A9C032025A926AA29AB0194ECE7259D0A9CBE
:20B88000002D149563DDB4BB099DE80733D4149C24EAE4739CE6299B7AE60DF1AA023E4D97
:20B8A000CB1785FB0150C3EBA00000EB8003A1EB43010928134601F130021A70014603F1D6
:20B8C000FF32ECDC00F130010DF1AB04C9B2944203F8011C5AD90DF19D001A4601E012F81E
:20B8E000011BA24200F8011FF9D10DF5907CC3EB4C03F63B72E70A9D6C1C149D2C4424EA73
:20B90000E47365E6DDE9200100220023FDF71CFB00287FF44AAFC5F1010525952C4424E6CA
:20B92000149D4FF067086C1C24EAE47350E6109DDDF840C02D680CF10403002D99F801802B
:20B940000A9510938146BEF615AEFEF710BE7CB9099DE9070CD401231C4639E6DDF824C09B
:20B960001CF001037FF443AF149324EAE4732FE60A9DAC1C24EAE4732AE60D9D0C232B60E9
:20B980004FF0FF30FEF7BABE259B13E70DF19E0324E700BF98F2000867666666024B13B16D
:20B9A000024800F07DB870470000000019CA00082DE9F04F384B85B01B68029003F5A47246
:20B9C00001930F460392019BD3F84881B8F1000F1CD0DDF80CB04FF00109DA46D8F8043017
:20B9E0005C1E11D408F188059E1C05EB830508EB860677B1EB6FBB420BD0013C631CA5F105
:20BA00000405A6F10406F4D1244A7ABB05B0BDE8F08FD8F8042056F8043C013AA24216BFC5
:20BA20000022C8F8044046F8042C002BE5D009FA04F2D8F88811D8F804B00A4210D0D8F8B0
:20BA40008C110A420ED1029855F8041C9847D8F804305B45B7D1DAF800304345CDD0B2E74C
:20BA60009847F4E755F8040C9847F0E7D8F804306BB9D8F8003063B14046CAF80030FEF750
:20BA80004DF9DAF80080B8F1000FA7D1BEE7D8F80030C2469846F6E74CF200081D9D00086E
:20BAA000014600200246034601F0C0BC2DE9F04F03690D6983B09D42834600F38C80013DD2
:20BAC00001F1140400F1140A54F825205AF825300132B3FBF2F8AA00914600925244A144BC
:20BAE0000192B8F1000F3ED000263046224653468C4652F8047B19681FFA87FE3F0C0EFB42
:20BB0000086E07FB08F606EB1E461FFA8EFECEEB000E8FB2B0B27744C0EB114000EB274042
:20BB2000BFB247EA0047914543F8047B4FEA20404FEA1646DDD2009A61465AF8023093B99E
:20BB4000019A131F9A450CD252F8043C4BB9A2F1080302E01A68043B1AB99A4505F1FF35B0
:20BB6000F8D3CBF81050584601F0F2FA00282EDB08F101085346002254F8046B1868B1B2D0
:20BB8000511A87B2360C3944C6EB104000EB214289B241EA0241A14543F8041B4FEA22426D
:20BBA000EAD25AF825200AEB850382B91A1F92450BD253F8042C42B9083B02E01A68043B31
:20BBC0001AB99A4505F1FF35F8D3CBF81050404603B0BDE8F08F002003B0BDE8F08F00BF88
:20BBE0002DE9F04F016C9BB0044692469B46279D41B1436C01229A404B608A6001F0B2F8A3
:20BC000000232364BBF1000FD94633DB00232B60A54B1A4609EA0303934214D050465946AD
:20BC200000220023FDF790F9804648B3269E289D01233360002D00F0CA809C482860013835
:20BC40001BB0BDE8F08F269D42F20F732B60BAF1000F00F0A5809648289E002EF0D0C37855
:20BC6000002B00F0B68000F10803289D2B601BB0BDE8F08F01232BF000492B60CB46C7E766
:20BC800019AA18AB8DE80C00204652465B4601F0EFFA5FEA19550A9040F08B80189F199D2B
:20BCA0006FF482633D449D42C0F295821F3305F212425B1B09FA03F32AFA02F243EA0200C0
:20BCC000FCF764FE0126013DB846A1F1F87116960022784BFCF71CFD6DA3D3E90023FCF732
:20BCE000CBFE6DA3D3E90023FCF714FD064628460F46FCF75BFE6AA3D3E90023FCF7BCFE94
:20BD000002460B4630463946FCF704FD06460F46FDF74CF939460790002230460023FDF702
:20BD20001DF9002840F02982079E162E00F222826149524601EBC6015B46D1E90001FDF726
:20BD40002BF9002800F04C82013E079600260E96C5EB0805013D069500F126820025089542
:20BD6000079E002EC0F21782069D0D963544002606950C96249D092D2DD8052DC4BF043D91
:20BD80002495249EC8BF0025A6F10203D8BF0125032B22D8DFE813F0B7039E02C0039A0476
:20BDA000464A434BC9F3130000280CBF1046184652E7CBF3130343F07F51CDF858805046AC
:20BDC000A5F2FF3541F44011DDF8608080E73C4836E7C31C49E7002524950025656429460B
:20BDE000204600F099FF4FF0FF390126099025952064CDF83C900B96199B002BC0F2D280CB
:20BE0000079E0E2E00F3CE802B4B03EBC603D3E90001CDE9040125990029C0F28083DDE9F9
:20BE2000042359465046FCF751FFFDF7BFF80546FCF7BCFDDDE90423FCF71EFE02460B462C
:20BE400050465946FCF764FC099A05F13003B9F1010F06460F46137002F1010B64D000225B
:20BE6000184BFCF709FE0022002306460F46FDF76BF8002840F08180DDF82480099DC844A4
:20BE8000DDE904AB05F10209039428E0AFF3008061436F63A787D23FB3C8608B288AC63F99
:20BEA000FB799F501344D33F0000F07FA1F20008C0F200080000F83FD0F20008B4F2000843
:20BEC000A0F2000800002440FCF7D6FD0022002306460F46FDF738F8002840F0C183524660
:20BEE0005B4630463946FCF7F1FEFDF75FF80546FCF75CFD52465B46FCF7BEFD02460B4668
:20BF000030463946FCF704FC05F1300EC14509F801EC4C4606460F464FF00002A74B09F1B1
:20BF20000109D1D1A346039C32463B4630463946FCF7F0FB06460F463246DDE904013B469C
:20BF4000FDF70CF840B9DDE9040132463B46FCF7FBFF90B1EB0710D51BF8015C099A05E02F
:20BF60009A4200F0298413F8015C9B46392D0BF1FF33F5D06A1CD2B21A7020460A9900F019
:20BF8000F1FE079E269D731C289E00228BF800202B60002E00F025830998C6F800B01BB005
:20BFA000BDE8F08F0B9D002D00F00381249E012E40F3DC820C9E09F1FF37BE42C0F28983FA
:20BFC000F71BB9F1000FC0F28784089D4B46089E20461E440896069E01211E44069600F0E3
:20BFE00063FF064665B10698002809DD03460899AB42A8BF2B46C91AC01A0891ED1A06902F
:20C000000C9A002A1DDD0B9B002B00F05883002F11DD31463A46204600F0EEFF06463146A0
:20C020000A9A204600F04AFF0A998046204600F099FECDF82880DDF830E0BEEB070240F033
:20C040008F822046012100F02FFF80460D98002805DD414620460D9A00F0CEFF80462499E0
:20C06000012940F3C18200270D98002840F0AF820120069B034413F01F0300F0A180C3F1D8
:20C080002002042A40F3B7840899069AC3F11C0319441A4408911D4406920899002905DDD5
:20C0A0000A99089A204600F0F5FF0A90069A002A04DD4146204600F0EDFF80460E9B002B49
:20C0C00040F06A82B9F1000F40F3A6820B98002840F088800B9D0A9FDDF824B006E03946CE
:20C0E00020460A22002300F047FE074638464146FFF7DCFC30300BF805000135A945EEDCE0
:20C10000DDF824B082460A97B9F1010FACBFCB440BF1010B00250A990122204600F0BAFFD7
:20C1200041460A9001F014F8002840F309831BF8012C099905E0994200F08B8213F8012C23
:20C140009B46392A0BF1FF33F5D001321A704146204600F007FE002E3FF40FAF2DB1B54215
:20C1600003D02946204600F0FDFD3146204600F0F9FD02E701260E96EAE50798FCF716FC43
:20C1800032463B46FCF7E0FE00287FF4CDAD079E013E0796C8E5079E089DAD1B089575422C
:20C1A00000260C950D96E5E56D42002608950696D6E50C9F089D0B9E14E700BF000024406B
:20C1C0001C23DDF820E006989E441844CDF820E01D44069061E7A748401B0AFA00F06FE5D9
:20C1E0000E90B5E5002D05DD31462A46204600F051FF0646002F40F0E9823746099D099891
:20C200004D4408950AF001050B95DDF82890451C0AE000F0B1FD394606460A22204600235A
:20C2200000F0AAFD0746013541464846FFF73EFC31468346484600F08BFF414603903A46BD
:20C24000204600F0A9FFC268691E03460BF1300A0691002A40F0938119464846029300F039
:20C2600077FF029B024619462046029200F07AFD029A2AB9249B1BB90B98002800F09383C0
:20C28000039B002BC0F2348205D1249818B90B99002900F02D82002A00F3AC82DDF820E07E
:20C2A00005F801AC7545AB4600F0B48249460A220023204600F060FDBE42814631462046CE
:20C2C0004FF00A024FF00003A3D100F055FD06460746A8E700260B96079EDDF894E0B64444
:20C2E0000EF10109B9F1000FCDF83CE04E4640F350810021172E61640AD9012204235B0050
:20C3000003F11400B042114602F10102F7D96164204600F001FD0E2E099020643FF66CAD46
:20C32000002D3FF469AD079DCDE912AB002D40F31C82514B05F00F0203EBC2032D11D3E923
:20C340000067EB0640F1CD814C4B50465946D3E90823FCF7BBFCCDE9100105F00F054FF09A
:20C3600003088DB1DFF814A130463946EE0705D5DAE9002308F10108FCF77EFB6D100AF158
:20C38000080AF3D106460F46DDE9100132463B46FCF79CFC82468B460E9D45B1504659465C
:20C3A0000022374BFCF7DAFD002840F0AA824046FCF7FCFA52465B46FCF75EFB0022314BF9
:20C3C000FCF7A8F90646A1F15077B9F1000F00F05A81079DC84617950B9D002D00F02382D8
:20C3E000254B002003EBC80353E902232649FCF76DFC32463B46FCF78BF9CDE910015946F2
:20C400005046FCF7D3FD0546FCF7D0FA02460B4650465946FCF77CF93035099ECDE90401BE
:20C42000DDE90423DDE91001EDB2357006F1010BFCF7B2FD002840F0AB82DDE904230020BD
:20C440000F49FCF765F902460B46DDE91001FCF7A3FD002840F0A282B8F1010F40F38181C6
:20C46000B044CDF85090A246C146DDE90467DDE9104519E0EEFBFFFFD0F2000898F30008AB
:20C480000000F03F00001C400000E03F0020A849FCF73EF922462B46FCF760FD002840F036
:20C4A0007B82CB4500F05A81204629460022A14BFCF7E2FA00229F4B04460D463046394654
:20C4C000FCF7DAFA0F460646FCF770FD8046FCF76DFA02460B4630463946FCF719F908F1E8
:20C4E00030085FFA88F822462B460BF8018B06460F46FCF733FD32463B460028C6D0179E93
:20C500005446079639E500260B96259800283CDD06460F908146ECE601260B96F5E7B9F12F
:20C52000000F3FF77CAC40F0C680DDE904010022814BFCF7A1FA52465B46FCF723FDC84677
:20C540004E4600287CD0259DDDF824B0ED4307954146204600F006FC002E7FF406AE0CE577
:20C560000A99204600F048FD0A906AE5169D002D00F0B88103F233430C9F089D27E501467D
:20C58000204600F0EFFB01227AE6012625960F96B14600216164BBE60A98414600F0D8FDE5
:20C5A0000028BFF68FADDDF81CE00A990EF1FF3E20460A220023CDF81CE000F0DDFB0A90DA
:20C5C0000B98002840F00982DDF83C907AE5D8F8103008EB8303186900F018FCC0F12000F6
:20C5E00047E50998FFF72CBBBAF1000F7FF43BADCBF31303002B40F07C812BF000473F0DA2
:20C600003F05002F3FF430AD089A069B0132013308920693012727E5249902297FF756AD25
:20C62000B9F1000F8FD141464B460522204600F0A3FB804641460A9800F08AFD002882DDC1
:20C64000079D312301350795099D2B7005F1010B7EE7079809993123013007900B7076E535
:20C66000A346039C89E44046FCF7A0F902460B4650465946FCF700FA0022304BFCF74AF826
:20C680000646A1F150775046594600222A4BFCF73FF832463B4682468B46FCF77DFC0028D9
:20C6A00040F0BD80324607F1004350465946FCF755FC002855D04FF00008464643E70A99F4
:20C6C0000C9A204600F098FC0A90BAE401260B9602E60C9D0D9E7B1B1E440C970D96002729
:20C6E0006FE4DDE912014FF00208CDE9100138E6002ACDF82890D94611DD0A990122204600
:20C7000000F0C8FC41460A9000F022FD002840F35D81BAF1390F00F01B8109F1310A069BA7
:20C72000354683F800A003F1010B3E460FE500BF0000F03F000024400000144000001C40E9
:20C7400003D11AF0010F7FF4F2AC5B4613F8012C9B46302A03F1FF33F8D0F8E4DDF8509047
:20C760005446DDE912ABFFF747BB079E7542002D00F0C280A34B05F00F0203EBC203D3E986
:20C780000023DDE91201FCF777F92D1182468B4600F02E819C4E4FF00208EA0705D5D6E907
:20C7A000002308F10108FCF767F96D1006F10806F3D182468B46EFE5079E099D30222A7017
:20C7C0000136312207961A70FFF7D7BB7168204600F0A2FA336905469A1C920006F10C0122
:20C7E0000C30FDF73FFD20462946012200F052FC074603E5BAF1390FCDF8289000F0A880DA
:20C80000069D0AF101032B703546069E06F1010B3E469CE43546CDF828903E467BE44FF09B
:20C82000000846460CE7774908F1FF3501EBC50132463B46D1E900011095FCF71DF9CDE9BA
:20C84000140159465046FCF7B1FB0546FCF7AEF802460B4650465946FBF75AFFDDF824E019
:20C860003035B8F1010F06460F468EF800500EF1010B1ED0099D6B1E03EB080A0022634B2B
:20C88000FCF7FAF80F460646FCF790FB8046FCF78DF808F1300802460B4630463946FBF7A5
:20C8A00037FF05F8018F5545E8D1109D06460F46AB440022564BDDE91401FBF72BFF3246F3
:20C8C0003B46FCF74BFB00284DD0179E099A07961BF8015CFFF74ABB089E0023C9EB060571
:20C8E000FFF775BB189B0C9FC3F13603089DFFF76EBB5746FFF7B8BBDDE912AB4FF0020831
:20C900004AE5B9F1000F3FF4AEAE0F9E002E7FF728AF00223D4B50465946FCF7ADF8824639
:20C9200008F101008B46FCF741F802460B4650465946FCF7A1F80022364BFBF7EBFE079D84
:20C940000646013DA1F150771795DDF83C8043E53546069B069E3922327003F1010B3E464E
:20C960000999FFF7EEBBDDE9142300202849FBF7CFFE32463B46FCF70FFB00283FF4F1AE39
:20C980005B4613F8012C9B46302A03F1FF33F8D0179D0795FFF7F1BA45465446179E099A27
:20C9A0000796FFF7E3BABAF1390FCDF82890CFD0039B3546002B069EC8BF0BF1310A86F814
:20C9C00000A006F1010B3E46FFF7C1BB7FF4A7AE1AF0010F3FF4A3AE9BE6314620460A22CE
:20C9E0000023DDF83C9000F0C7F90646FFF76ABB4FF00208D0E43FF450ABC3F13C03FFF748
:20CA0000E0BB00BFD0F2000898F30008000024400000E03F00001C4038B5094D094C641B69
:20CA2000A41018BF05EB840505D0013C55F8043D9847002CF9D1BDE8384000F0D5BF00BF1D
:20CA4000F4D90008F8D90008F8B5234D0F460446FDF7C8FCAB685E6826F00306F11B01F6B9
:20CA6000EF7121F47F6121F00F01A1F58057B7F5805F07DB20460021FDF7B8FCAB683344AD
:20CA8000984204D02046FDF7AFFC0020F8BD20467942FDF7ABFC01300DD0104BAA68196856
:20CAA000F61B46F001062046C91B56601960FDF79BFC0120F8BD20460021FDF797FCAB682D
:20CAC000C21A0F2ADEDD064D04492D6842F00102401B5A600860D5E7040B002088190020F3
:20CAE000100F00202DE9F0410D460646002955D0FDF778FC55F8041CDFF870C1A5F1080444
:20CB000021F00103E218DCF808005768904227F0030768D011F00101576032D00021D0197A
:20CB20004068C00706D43B44906800294DD0D268C260906043F001026260E350E1B9B3F536
:20CB4000007F2DD35A0A042A69D89809383041000CEB810CDCF808204449624565D0516897
:20CB600021F003018B4202D292689445F7D1D368E360A2609C60D4603046BDE8F041FDF774
:20CB800033BC55F8085C0CF10808641BA0682B44404542D0E568C560A860C0E7BDE8F08124
:20CBA000DB089A1001209040DCF804100CEBC3039A680143A260E360CCF8041030469C607D
:20CBC000D460BDE8F041FDF70FBC294DA842AED143F00102CCF81440CCF81040E060A0600B
:20CBE0006260E350C8E71F44CB0707D455F8081C641AE368A2680F44D3609A601D4B47F01E
:20CC000001021B6862609F42CCF80840B4D31A4B30461968FFF718FFAEE701217FE7142A94
:20CC20000BD802F15B00410092E780100125854048681346284348609AE7542A03D8180B75
:20CC40006E30410084E7B2F5AA7F03D8D80B773041007DE740F254518A4203D8980C7C30E2
:20CC6000410075E7FC217E2072E700BF040B00200C0B00200C0F00208419002000487047E7
:20CC8000140F0020830770B4C9B240D0541E2AB303788B4223D0431C04E0FCB105781446C7
:20CCA0008D421CD013F0030F184604F1FF3203F10103F2D1032C14D8651E54B303788B4278
:20CCC0000DD0421C002302E004788C4207D0AB42104603F1010302F10102F5D1002070BCB0
:20CCE000704741EA0126034646EA06461A6818467240A2F1013525EA020212F0803F03F143
:20CD00000403D9D1043C032C1846EFD8D4E71446D0E72046E3E700BFC26C70B505460C4623
:20CD20004AB152F8240080B1016842F8241000220261C26070BD2122042100F0CBFBE86444
:20CD400002460028EDD1002070BD012101FA04F6721D2846920000F0BDFB0028F3D044607B
:20CD60008660E4E731B1C36C4A6853F82200086043F82210704700BF2DE9F0430F6983B093
:20CD80008846814601F1140500242E680134B1B2360C02FB013302FB06F699B206EB1343A3
:20CDA00001EB0341A74245F8041B4FEA1343ECDC4BB1D8F80820974209DA08EB8702013743
:20CDC0005361C8F81070404603B0BDE8F083D8F80410484601310193FFF79EFFD8F8102043
:20CDE00008F10C010232044692000C30FDF73AFAD9F84C20D8F80410019B52F82100C8F8D1
:20CE0000000042F82180A046D7E700BF030C1B04B3B90004102310F07F4F04BF0002083335
:20CE200010F0704F04BF0001043310F0404F04BF80000233002807DB420003D42020704717
:20CE40000023E8E7581C704718467047036813F0070207D0D90720D49A0720D49B080360E3
:20CE60000220704799B209B91B0C102213F0FF0F04BF1B0A0832190704BF1B090432990763
:20CE800004BF9B080232D90704D45B0801D1202070470132036010467047002070475B0837
:20CEA00003600120704700BF10B50C460121FFF733FF01224461026110BD00BF2DE9F04F0B
:20CEC0000D69D2F8109085B04D450C46924604DA2A4654464D468A469146A36805EB090754
:20CEE00061689F42C8BF0131FFF716FF00F1140606EB87084645019005D23346002043F872
:20CF0000040B9845FBD80AF1140C0CEB89091434CC45009404EB85055BD2CDF80880039734
:20CF2000C8465CF8043B9CB224B3009A33464FF0000900E00B4652F8047B19681FFA87FBBA
:20CF40001FFA81FA380C090C04FB0BAA04FB0010D14400EB19401FFA89F949EA0047194654
:20CF600095424FEA104941F8047BE3D8C3F804905CF8043C5FEA134924D0D6F800A0009B50
:20CF8000504631464FF0000B00E011461A88000C09FB02001FFA8AFA83444AEA0B400A461C
:20CFA00042F8040B53F8047B48684FEA174A84B209FB0A4A9D420AEB1B4A4FEA1A4BE4D8F3
:20CFC000C1F804A0E04506F10406AAD8DDF80880039F002F0ADD58F8043CA8F104081BB136
:20CFE00004E058F8043D0BB9013FFAD1019B18461F6105B0BDE8F08F12F003032DE9F0414B
:20D00000144607460E462CD1A4101CD0BD6C002D30D04FF0000804E0641014D02868A8B1B6
:20D020000546E307F8D5384631462A46FFF746FFAEB17268FB6C641053F82210316043F8F1
:20D0400022600646EAD13046BDE8F081384629462A46FFF733FF2860C0F80080E0E7064663
:20D06000DAE70B4A013B52F823200023FFF784FE0646C9E701213846FFF74EFE40F2712194
:20D0800001220023416102610546B8640360C0E7C0F300082DE9F84F0B694FEA621A0AEB9E
:20D0A00003098B6809F101069E420F4693468046496804DD5B009E4201F10101FADC40467F
:20D0C000FFF72AFEBAF1000F00F1140409DD00231A4625460133534545F8042BFAD104EBA9
:20D0E00083043A6907F114031BF01F0B03EB820C21D0CBF1200A002200E02C46196825460F
:20D1000001FA0BF10A4345F8042B53F8042B634522FA0AF2F1D362600AB109F10206D8F812
:20D120004C307A68013E53F822100661396043F82270BDE8F88F53F8042B9C4544F8042B16
:20D14000EDD953F8042B9C4544F8042BF3D8E6E702690B6910B4D21A15D19B001430143112
:20D160001944034401E0984211D253F8042D51F8044DA242F7D0944294BF01204FF0FF30F4
:20D180005DF8044B704710465DF8044B704700205DF8044B704700BF2DE9F0470D4604465F
:20D1A000114628461646FFF7D3FF071E56D04FDB4FF0000969682046FFF7AEFD2F693269BE
:20D1C00014351436C0F80C9000F1140305EB870C06EB8208002155F8044B56F8042B1FFA0F
:20D1E00084FA8A441FFA82F9110CC1EB1441C9EB0A0201EB224192B242EA0142B04543F83F
:20D20000042B4FEA21412C46E5D8AC45984615D954F8046BB2B21144360C06EB214689B20F
:20D2200041EA0642A44543F8042B4FEA2641EFD8EB43634423F0030304334344043B22B9FB
:20D2400053F8042D013F002AFAD00761BDE8F0872B464FF0010935461E46ABE7204639468A
:20D26000FFF75AFD012347610361BDE8F08700BF2DE9F043012183B01D46C3F30A561446E5
:20D280000A9FFFF749FDC5F3130380460EB143F48013019324B302A840F8084D6846FFF746
:20D2A000D5FD002835D19DE80C00C8F81420002B0CBF01240224C8F81830C8F81040DEB9F9
:20D2C00008EB8403A0F2324038601869FFF79EFD0B9BC0EB44101860404603B0BDE8F083B8
:20D2E00001A8FFF7B3FD019B01242030C8F81430C8F81040002EE3D0A6F2334909EB0003CE
:20D300003B600B9BC0F135001860404603B0BDE8F083019BC0F1200103FA01F1C340009A23
:20D3200001930A43C8F81420C1E700BF2DE9F04F946883B0924680460D461668002C6FD053
:20D340004FF0000B08688B685C46002C43D09C421F4645D3AB8913F4906F44D06F6929692C
:20D3600007EB470707EBD777C1EB0009621C7F104A44974234BF17463A465B0535D5114673
:20D380004046FCF7D3FC002839D029694A460190FCF768FFAA89019B22F4906242F080027C
:20D3A000AA81C9EB070203EB09006F612B612860AA602746A1464A46594600F0BBF8DAF8A8
:20D3C0000820AB682868DB1B4844141BAB602860CAF8084024B3D6F800B074680836B4E72A
:20D3E0002746A146E7E7B946E5E7404600F008F903460028D5D140462969FFF773FBAA8903
:20D400000C23C8F8003042F0400200234FF0FF30AA81CAF80830CAF8043003B0BDE8F08FF6
:20D420002046CAF8044003B0BDE8F08FF0B5274C85B026680746D6F84841002C40D0656821
:20D440001F2D1EDD224818B94FF0FF3005B0F0BD4FF4C870039102920193FCF757FC039961
:20D460000446029A019B0028EED0D6F848510020256060600546C6F84841C4F88801C4F8E5
:20D480008C013FB96B1C00200235636044F8251005B0F0BD0126AE4004EB8500C0F88820AA
:20D4A000D4F88821022F42EA0602C4F88821C0F80831E7D1D4F88C311E43C4F88C61E1E729
:20D4C00006F5A674C6F84841B9E700BF4CF200080D9D000810B502FB01F1FCF727FC044685
:20D4E00068B150F8042C22F00302043A242A18D8132A06D8034600221A605A609A602046EE
:20D5000010BD00231B2A036043600FD9242A8360C36005BF0361436100F1100300F11803B8
:20D52000E9E70021FCF714FF204610BD00F10803E1E700BF8842F0B410D98C18A0420DD282
:20D540008518531E42B121462A4611F8014D013B02F8014D5C1CF8D1F0BC70470F2A44D91E
:20D5600040EA01039B0744D1A2F110073F0900EB071610360C4603462568103343F8105C74
:20D580006568103443F80C5C54F8085C43F8085C54F8045C43F8045CB342EDD17B1C02F005
:20D5A0000F0C1B01BCF1030F1944034423D90E461D46644656F8047B043C032C45F8047B7C
:20D5C000F8D8ACF1040424F00304043402F0030223442144002ABFD01A4411F8014B03F859
:20D5E000014B9342F9D1F0BC70470346002AF3D1B2E70346F0E76246002AEDD1ACE700BF0B
:20D600002DE9F04F0C4683B090468146002900F0BA80FCF7E7FE08F10B0654F8043C162E8E
:20D6200023F00305A4F108074BD810210E46B0454CD88D4251DADFF884B37819DBF808E016
:20D64000864500F0A680426822F0010C8444DCF804C01CF0010F54D000221046DB076FD4E3
:20D6600054F8083CC3EB070ADAF8043023F003032B44002862D0704500F0E98002EB030E67
:20D680008E455BDBC3688268D046D3609A6058F8081FDAF80C302A1F242ACB60996000F2F7
:20D6A0002381132A40F2B08023681B2ACAF808306368CAF80C3000F22B8108340AF11003AC
:20D6C000A3E026F00706002E3146B0DA0C230020C9F8003003B0BDE8F08FA046AA1B0F2A7A
:20D6E00003F001031AD82B437B603D446B6843F001036B604846FCF777FE404603B0BDE8CE
:20D70000F08F22F0030202EB050C8C45A6DBC2688168A046CA6065469160DFE7B919334356
:20D7200042F001007B600A4448605368083143F0010353604846FFF7D5F9DBE78B4233DA19
:20D7400041464846FCF7F2FA80460028D2D054F8043CA0F1080123F001023A44914200F0C8
:20D76000BC802A1F242A6ED8132A42D803462246116819605168596092689A60214648463B
:20D78000FFF7B0F9B6E7114603B0BDE8F04FFCF7CDBADEF8042006F1100C22F00302501958
:20D7A00060453DDA704659E7D04658F8080FDAF80C102A1F242AC160886000F2A080132A5D
:20D7C00040F29B8021681B2ACAF808106168CAF80C1000F2B28008340AF1100221681D4654
:20D7E0001160616857465160A3689360DAF8043074E723681B2A03606368436062D800F176
:20D80000080304F10802B3E74346226875461A60626857465A60A2689A60DAF804305DE7AD
:20D82000831B374443F00103CBF808707B6054F8043C484603F001031E4344F8046CFCF771
:20D84000D3FD20465AE72146FFF774FE96E702EB030C06F110029445FFF670AF574657F827
:20D86000081FDAF80C302A1F242ACB60996000F28680132A77D923681B2ACAF8083063689E
:20D88000CAF80C3000F2848008340AF1100322681A6062685A60A2689A60C6EB0C020AEB0A
:20D8A000060342F00102CBF808305A60DAF80430484603F001031E43CAF80460FCF794FDDF
:20D8C00038461BE7A368242A8360E368C3602BD000F1100304F110024AE750F8042CA04689
:20D8E00022F003021544F9E62146404675465746FFF720FEDAF80430F0E642466EE7214660
:20D9000040461D465746FFF715FEDAF80430E5E6A368242ACAF81030E368CAF8143018D013
:20D9200010340AF1180370E7226900F118030261616904F1180241611AE7A168242ACAF8A7
:20D940001010E168CAF814100FD010340AF1180244E722690AF12003CAF81820626918345B
:20D96000CAF81C2051E73B4691E721690AF12002CAF8181061691834CAF81C102EE7214667
:20D980003846CDF804C0FFF7D5FDDDF804C084E7A368242ACAF81030E368CAF8143003D035
:20D9A00010340AF1180372E722690AF12003CAF8182062691834CAF81C2068E7040B00207E
:20D9C000F8B500BFF8BC08BC9E4670479DB90008F56A0008112100081931000849460008E0
:20D9E0008D4B0008A96C0008F8B500BFF8BC08BC9E467047ED200008D470FF7F01000000D3
:20DA0000000000000000000020212223242526270001020304050607101112131415161732
:20DA200018191A1B1C1D1E1F2C00C20100000008020300004200000059310008000000003A
:20DA4000E9310008000000000000000000000000913200084D3200085C0000201932000883
:20DA6000000000004000000800000000000000001000000BE53200080000000040000000E4
:20DA8000400000004000000000030000000000000000000000000000000000000000000003
:20DAA000000000000000000000000000000000000000000000000000000000000000000066
:20DAC000000000000000000000000000000000000000000000000000000000000000000046
:20DAE000000000000000000000000000000000000000000000000000000000000000000026
:20DB0000000000000000000000000000000000000000000000000000000000000000000005
:20DB2000A812002000000000320100201200000000011201000200000140AF1E240000025C
:20DB400001020001F40100007CEC00080400000040EC0008000000000CEC00080000000024
:20DB60000000000000000000030000008800002000000000000000020004000601010000EC
:20DB800019000000A541000800000000A5400008000000000000000075420008F940000891
:20DBA00001420008A8010020C5400008000000004000000B4000000089EC00080900000033
:20DBC000ACEC0008050C0901A1018503150026FF0319002AFF03751095018100C000000082
:20DBE0009CEC0008A4EC0008B4EC000805010902A10185010901A100050919012908150003
:20DC0000250195087501810205010930093109381581257F750895038106C0C00501090425
:20DC2000A101851415002501750195200509190129208102150025073500463B0175049549
:20DC400001651405010939814205010901A100150026FF03750A950409300931093309344D
:20DC60008102C0150026FF03750A9502093609368102C005010906A1018502050719E029E1
:20DC8000E7150025017501950881029501750881039506750815002565050719002965814A
:20DCA00000050819012908950875019102C00000000010000500008000000100B00200203E
:20DCC000002801400100000000240140001200000000000000000000000000000000000063
:20DCE000C0020020C80200200000024007000000000000000B000000000000000C000000F8
:20DD0000000000000D000000000000000E000000000000000F0000000000000010000000C9
:20DD20000000000011000000E8020020000801400B000000000C01400C01000000100140C9
:20DD40000D020000001401400E030000005400400000000000000000000000003403002063
:20DD6000000000000000000000000706121F20000000000000000000000000000000000045
:20DD8000000000000058004000000000000000000000000034030020000000000000000094
:20DDA00000000B0A1321220000000000000000000000000000000000000000001C1002408A
:20DDC0001810024014100240101002400C1002401C10024018100240141002400004004031
:20DDE0001C0100000000000000000000000000000000000000000000000000000000000006
:20DE0000000800401D0100000000000000000000000000000000000000000000000000009C
:20DE200000000000002C01401A00000000000000000000000000000000000000000000005B
:20DE4000000000000000000000000000000000401B01000000000000000000000000000066
:20DE6000000000000000000000000000000000007C04002010050020A4050020003801408B
:20DE80000C1700200017002020AA44000000000000000000000000000000000000000000FA
:20DEA000000000000000000000000000000000000000000000000000000000000000000062
:20DEC000000000000000000000000000000000000000000000000000000000000000000042
:20DEE000000000000000000000000000000000000000000000000000000000000000000022
:20DF00000000000000000000000000002825000000440040181700203017002010552200F3
:20DF20000000000000000000000000000000000000000000000000000000000000000000E1
:20DF40000000000000000000000000000000000000000000000000000000000000000000C1
:20DF60000000000000000000000000000000000000000000000000000000000000000000A1
:20DF8000000000000000000000000000000000000000000000000000000000000000000081
:20DFA0002926000000480040241700203C1700201055220000000000000000000000000035
:20DFC000000000000000000000000000000000000000000000000000000000000000000041
:20DFE000000000000000000000000000000000000000000000000000000000000000000021
:20E00000000000000000000000000000000000000000000000000000000000000000000000
:20E0200000000000000000000000000000000000000000002A2700003C06002000BF00006E
:20E04000000000000000000000002D0040F1000843000000215C0008055D00089567000824
:20E0600095670008095B00085D5B0008AD5B0008155C0008095C0008E95B0008000000002E
:20E080004000000083F10008040000001CF100081200000010F100080C00000000C20100C1
:20E0A0000000080095670008BD5B0008956700089567000895670008956700089567000820
:20E0C00095670008D95B00082EF1000812000000040101000000000000000000C4090020D4
:20E0E0002C0A0020940A00200000000000000000000000000000000000000000000000000C
:20E1000000000000000000000000000048F2000800000000000000000000000000000000BD
:20E120000000000000000000000000000000000000000000000000000000000000000000DF
:20E140000000000000000000000000000000000000000000000000000000000000000000BF
:20E1600000000000000000000000000000000000000000000000000000000000000000009F
:20E1800001000000000000000E33CDAB34126DE6ECDE05000B000000000000000000000052
:20E1A00000000000000000000000000000000000000000000000000000000000000000005F
:20E1C00000000000000000000000000000000000000000000000000000000000000000003F
:20E1E00000000000000000000000000000000000000000000000000000000000000000001F
:20E200000000000000000000000000000000000000000000000000000000000000000000FE
:20E220000000000000000000000000000000000000000000000000000000000000000000DE
:20E240000000000000000000000000000000000000000000000000000000000000000000BE
:20E2600000000000000000000000000000000000000000000000000000000000000000009E
:20E2800000000000000000000000000000000000000000000000000000000000000000007E
:20E2A00000000000000000000000000000000000000000000000000000000000000000005E
:20E2C00000000000000000000000000000000000000000000000000000000000000000003E
:20E2E00000000000000000000000000000000000000000000000000000000000000000001E
:20E300000000000000000000000000000000000000000000000000000000000000000000FD
:20E320000000000000000000000000000000000000000000000000000000000000000000DD
:20E340000000000000000000000000000000000000000000000000000000000000000000BD
:20E3600000000000000000000000000000000000000000000000000000000000000000009D
:20E3800000000000000000000000000000000000000000000000000000000000000000007D
:20E3A00000000000000000000000000000000000000000000000000000000000000000005D
:20E3C00000000000000000000000000000000000000000000000000000000000000000003D
:20E3E00000000000000000000000000000000000000000000000000000000000000000001D
:20E400000000000000000000000000000000000000000000000000000000000000000000FC
:20E420000000000000000000000000000000000000000000000000000000000000000000DC
:20E440000000000000000000000000000000000000000000000000000000000000000000BC
:20E4600000000000000000000000000000000000000000000000000000000000000000009C
:20E4800000000000000000000000000000000000000000000000000000000000000000007C
:20E4A00000000000000000000000000000000000000000000000000000000000000000005C
:20E4C00000000000000000000000000000000000000000000000000000000000000000003C
:20E4E00000000000000000000000000000000000000000000000000000000000000000001C
:20E50000D80600200000000000000000040B0020040B00200C0B00200C0B0020140B0020F2
:20E52000140B00201C0B00201C0B0020240B0020240B00202C0B00202C0B0020340B002063
:20E54000340B00203C0B00203C0B0020440B0020440B00204C0B00204C0B0020540B002043
:20E56000540B00205C0B00205C0B0020640B0020640B00206C0B00206C0B0020740B002023
:20E58000740B00207C0B00207C0B0020840B0020840B00208C0B00208C0B0020940B002003
:20E5A000940B00209C0B00209C0B0020A40B0020A40B0020AC0B0020AC0B0020B40B0020E3
:20E5C000B40B0020BC0B0020BC0B0020C40B0020C40B0020CC0B0020CC0B0020D40B0020C3
:20E5E000D40B0020DC0B0020DC0B0020E40B0020E40B0020EC0B0020EC0B0020F40B0020A3
:20E60000F40B0020FC0B0020FC0B0020040C0020040C00200C0C00200C0C0020140C00207D
:20E62000140C00201C0C00201C0C0020240C0020240C00202C0C00202C0C0020340C00205A
:20E64000340C00203C0C00203C0C0020440C0020440C00204C0C00204C0C0020540C00203A
:20E66000540C00205C0C00205C0C0020640C0020640C00206C0C00206C0C0020740C00201A
:20E68000740C00207C0C00207C0C0020840C0020840C00208C0C00208C0C0020940C0020FA
:20E6A000940C00209C0C00209C0C0020A40C0020A40C0020AC0C0020AC0C0020B40C0020DA
:20E6C000B40C0020BC0C0020BC0C0020C40C0020C40C0020CC0C0020CC0C0020D40C0020BA
:20E6E000D40C0020DC0C0020DC0C0020E40C0020E40C0020EC0C0020EC0C0020F40C00209A
:20E70000F40C0020FC0C0020FC0C0020040D0020040D00200C0D00200C0D0020140D002074
:20E72000140D00201C0D00201C0D0020240D0020240D00202C0D00202C0D0020340D002051
:20E74000340D00203C0D00203C0D0020440D0020440D00204C0D00204C0D0020540D002031
:20E76000540D00205C0D00205C0D0020640D0020640D00206C0D00206C0D0020740D002011
:20E78000740D00207C0D00207C0D0020840D0020840D00208C0D00208C0D0020940D0020F1
:20E7A000940D00209C0D00209C0D0020A40D0020A40D0020AC0D0020AC0D0020B40D0020D1
:20E7C000B40D0020BC0D0020BC0D0020C40D0020C40D0020CC0D0020CC0D0020D40D0020B1
:20E7E000D40D0020DC0D0020DC0D0020E40D0020E40D0020EC0D0020EC0D0020F40D002091
:20E80000F40D0020FC0D0020FC0D0020040E0020040E00200C0E00200C0E0020140E00206B
:20E82000140E00201C0E00201C0E0020240E0020240E00202C0E00202C0E0020340E002048
:20E84000340E00203C0E00203C0E0020440E0020440E00204C0E00204C0E0020540E002028
:20E86000540E00205C0E00205C0E0020640E0020640E00206C0E00206C0E0020740E002008
:20E88000740E00207C0E00207C0E0020840E0020840E00208C0E00208C0E0020940E0020E8
:20E8A000940E00209C0E00209C0E0020A40E0020A40E0020AC0E0020AC0E0020B40E0020C8
:20E8C000B40E0020BC0E0020BC0E0020C40E0020C40E0020CC0E0020CC0E0020D40E0020A8
:20E8E000D40E0020DC0E0020DC0E0020E40E0020E40E0020EC0E0020EC0E0020F40E002088
:20E90000F40E0020FC0E0020FC0E002000000200FFFFFFFFCCF2000880F2000880F20008C9
:20E9200080F2000880F2000880F2000880F2000880F2000880F2000880F20008FFFFFFFF85
:20E94000FFFFFFFFFFFFFFFFFFFF0000000000002564202564204D256420707265737365E7
:20E96000640A002564202564204D25642072656C65617365640A004225642070726573737A
:20E9800065640A0066616C7365207363726F6C6C65640A0074727565207363726F6C6C6543
:20E9A000640A00436C6F636B776F726B5049004465765465726D003230323130353331005C
:20E9C000736574757020646F6E650000EA00EB00EC00ED00EE00EF00F000F1008100F20061
:20E9E000800087008200F300F400F500FA00050C0901A1018503150026FF0319002AFF03F1
:20EA0000751095018100C005010906A1018502050719E029E71500250175019508810295E1
:20EA20000175088103950675081500256505071900296581000508190129089508750191ED
:20EA400002C005010904A101851415002501750195200509190129208102150025073500D6
:20EA6000463B0175049501651405010939814205010901A100150026FF03750A9504093042
:20EA80000931093309348102C0150026FF03750A9502093609368102C005010902A1018534
:20EAA000010901A1000509190129081500250195087501810205010930093109381581250B
:20EAC0007F750895038106C0C000E800E900F80060005B005D002D003D00310032003300BA
:20EAE0003400350036003700380039003000B100B300DA00D900D800D7007100770065008C
:20EB0000720074007900750069006F0070006100730064006600670068006A006B006C002B
:20EB20007A0078006300760062006E006D002C002E002F005C003B002700B200B00086009E
:20EB4000840085002000FFFFFFFFCE00D000F90060005B005D00CC00CD00C200C300C400FF
:20EB6000C500C600C700C800C900CA00CB00B100C100D300D600D200D5007100770065000E
:20EB80007200740079007500D1006F0070006100730064006600670068006A006B006C0043
:20EBA0007A0078006300760062006E006D00F700F6002F005C003B002700D400B000860069
:20EBC000840085002000FFFFFFFF080B0002020201020904000001020201000524000110A7
:20EBE0000524010301042402060524060001070580031000FF09040100020A0000000705C3
:20EC00000002400000070580024000004D61706C650009020000000100C0320095670008F3
:20EC2000AD360008956700089567000895670008ED36000895670008956700081537000856
:20EC40004C6561664C61627300000000BD370008453800089567000895670008D93500081B
:20EC60004536000825370008B1370008A53700084137000800000000400000000403090405
:20EC80000904000001030100000921100100012200000705800340000A0000001C020020ED
:20ECA00057000000730200203B000000C401002019000000EC0100203000000000000000F2
:20ECC000000000002A2B280000000000000000000000000000000000000000002C9EB4A099
:20ECE000A1A2A434A6A7A5AE362D3738271E1F20212223242526B333B62EB7B89F848586C7
:20ED00008788898A8B8C8D8E8F909192939495969798999A9B9C9D2F3130A3AD35040506B1
:20ED20000708090A0B0C0D0E0F101112131415161718191A1B1C1DAFB1B0B5000000000070
:20ED40000000000000000000C1430008596A0008396A000845440008A3440008A1430008C5
:20ED60000000000000000000454800085D480008396A000881460008A34600088546000813
:20ED8000E5470008000000002C0300204C040020C8020020000100002C0300204C040020D6
:20EDA000C8020020010201002C0300204C040020C8020020020302002C0300204C040020F6
:20EDC000C8020020030403002C03002000000000C8020020040004002C03002000000000AF
:20EDE000C8020020050005002C030020DC030020C8020020060106002C030020DC0300208C
:20EE0000C8020020070207002C03002024040020000000000801FF002C03002024040020C2
:20EE2000000000000902FF002C03002024040020000000000A03FF002C030020240400208E
:20EE4000000000000B04FF002C03002000000000000000000C00FF002C03002000000000FB
:20EE6000000000000D00FF002C03002000000000000000000E00FF002C03002000000000DB
:20EE8000000000000F00FF0034030020DC030020C80200200003080034030020DC030020C3
:20EEA000C8020020010409003403002000000000000000000200FF003403002000000000AB
:20EEC000000000000300FF003403002000000000000000000400FF0034030020000000007F
:20EEE000000000000500FF003403002000040020000000000601FF00340300200004002012
:20EF0000000000000702FF003403002000040020000000000803FF003403002000040020E9
:20EF2000000000000904FF003403002000000000000000000A00FF0034030020000000000E
:20EF4000000000000B00FF003403002000000000000000000C00FF003403002000000000EE
:20EF6000000000000D00FF003403002000000000000000000E00FF003403002000000000CA
:20EF8000000000000F00FF003C03002000000000C802002000000A003C03002000000000B1
:20EFA000C802002001000B003C03002000000000C802002002000C003C03002000000000A5
:20EFC000C802002003000D003C03002000000000C802002004000E003C030020000000007D
:20EFE000C802002005000F003C03002000000000000000000600FF003C0300200000000050
:20F00000000000000700FF003C03002000000000000000000800FF003C0300200000000025
:20F02000000000000900FF003C03002000000000000000000A00FF003C0300200000000001
:20F04000000000000B00FF003C03002000000000000000000C00FF003C03002000000000DD
:20F06000000000000D00FF003C03002000000000000000000E00FF003C03002000000000B9
:20F08000000000000F00FF004403002000000000000000000200FF002C0300203403002054
:20F0A0000109010A010F0100001B02060000020000000204000001020103010401050000ED
:20F0C0000000000000150016001C0000010C000E00000202010B00000001000200000000BB
:20F0E00000000000000000000000000000000000010E00110012000000000017F0000000D7
:20F1000000070000003800000000C00000C000000C034D00610070006C00650012034C00D1
:20F120006500610066004C006100620073001201000202000040AF1E0400000201020001F3
:20F1400009024300020100C0320904000001020201000524000110052401030104240206C1
:20F160000524060001070582034000FF09040100020A000000070503024000000705810295
:20F1800040000004030904000000000000000000FD690008596A0008396A0008B569000811
:20F1A0007B690008C1690008E3690008000000000000000000000000B76A0008596A0008E9
:20F1C000396A0008000000000000000000000000416C0008576C0008396A0008A16B000845
:20F1E000C36B0008A56B00088D6C000800000000706F7700737172740000000073717274D6
:20F20000660000000000000000000000000000000000004003B8E23F00000000000000006C
:20F2200006D0CF43EBFD4C3E000000000000F03F000000000000F83F00000000000030439B
:20F2400000000000000030C343000000D8060020303030303030303030303030303030307A
:20F26000494E4600696E66004E414E006E616E0030313233343536373839414243444546B8
:20F28000000000003031323334353637383961626364656600000000286E756C6C29000000
:20F2A0003000000020202020202020202020202020202020496E66696E69747900000000D4
:20F2C0004E614E00504F5349580000002E000000000000000000F03F0000000000002440DD
:20F2E00000000000000059400000000000408F40000000000088C34000000000006AF84039
:20F300000000000080842E4100000000D01263410000000084D797410000000065CDCD4181
:20F32000000000205FA00242000000E876483742000000A2941A6D42000040E59C30A24277
:20F340000000901EC4BCD64200003426F56B0C430080E03779C3414300A0D88557347643C6
:20F3600000C84E676DC1AB43003D9160E458E143408CB5781DAF154450EFE2D6E41A4B44C4
:20F3800092D54D06CFF08044F64AE1C7022DB544B49DD9794378EA440080E03779C341433D
:20F3A000176E05B5B5B89346F5F93FE9034F384D321D30F94877825A3CBF737FDD4F157525
:20F3C00005000000190000007D00000000DA0008FFFFFFFFFFFFFFFFFFFFFFFFFFFFFFFFC0
:20F3E000FFFFFFFFFFFFFFFFFFFFFFFFFFFFFFFFFFFFFFFFFFFFFFFFFFFFFFFFFFFFFFFF2D
:20F40000FFFFFFFFFFFFFFFFFFFFFFFFFFFFFFFFFFFFFFFFFFFFFFFFFFFFFFFFFFFFFFFF0C
:20F42000FFFFFFFFFFFFFFFFFFFFFFFFFFFFFFFFFFFFFFFFFFFFFFFFFFFFFFFFFFFFFFFFEC
:20F44000FFFFFFFFFFFFFFFFFFFFFFFFFFFFFFFFFFFFFFFFFFFFFFFFFFFFFFFFFFFFFFFFCC
:00000001FF
